:1061C90001190000090101240200000301FA040079
:1061D900FA0500030A0A5A0B001E0C00FA0D000307
:1061E9000E00040F0164100096120132130AFA140A
:1061F900010215000217010A1801FA1905321A01DC
:106209000A1B01FA1C05321FFFFF20FFFF23011E95
:106219002400642A00FA2B00FA2C50782D003D2E18
:1062290000462F001E3000643250783300003432AB
:10623900FA350164360164370150380A643C006458
:106249003E003C3F000140FFFF411450420A5A43BF
:106259000AC84405324500B44600FA4701484802D5
:10626900034C00FA4EFFFF500404510596520A32BE
:10627900530B46540A9656010257054658000259CF
:106289000A465A32FA5B010A5C0A325E000A5F006A
:10629900FE61FFFF64021166000267FFFF6A0A3CA4
:1062A9006B00006C3296730000740000780132793B
:1062B90001327EFFFF81FFFF84FFFF8500AF86006B
:1062C900018700FA89010A8A00009900009D0A964F
:1062D9009E00019FFFFFA0FFFFFAFAFA00000901E3
:1062E90001240200000301FA0400FA0500030A0A66
:1062F9005A0B001E0C00FA0D00030E00040F016476
:10630900100096120132130AFA140102150000173F
:10631900010A1801FA1905321A010A1B01FA1C05AA
:10632900321FFFFF20FFFF23011E2400642A00FA09
:106339002B00FA2C50782D003D2E00462F001E30E0
:1063490000643250783300003432FA350164360182
:1063590064370150380A643C00643E003C3F000148
:1063690040FFFF411450420A5A430AC844053245C6
:1063790000B44600FA4701244802024C00FA4EFFD5
:10638900FF500404510596520A32530B46540A969B
:10639900560101570546580001590A465A32FA5B17
:1063A900010A5C0A325E000A5F00FE61FFFF6402B7
:1063B9001166000267FFFF6A0A3C6B00006C3296A7
:1063C9007300007400007801327901327EFFFF8189
:1063D900FFFF84FFFF85FFFF86FFFF87FFFF89011E
:1063E900028A00009900009D0A969E00019FFFFF06
:1063F900A0FFFFFAFAFA0065006F00790083008DAB
:10640900009700A100AC00B600C000CA00D400DEAD
:1064190000E800F200580060006800700078008011
:1064290000880090009800A000A800B000B800C142
:1064390000C800D000D800DF00E600EE00F60041F9
:106449000047004D00530059005F0065006C007162
:106459000077007D00830089008F0095009B00A2D2
:1064690000A700AC00B200B900C000C500CA00D244
:0A64790000D500DD00E100E700EFB0
:103A3900900049E0D3940440149007BAE0FEA3E053
:103A4900FF9061CB1265BCE493F59980129007BA97
:103A5900E0FEA3E0FF9062E51265BCE493F599905E
:103A690007BAE0FEA3E0FF9061C9E493FC740193F7
:103A7900FDEFB50507EEB50403754D009007BA12C1
:103A890065A32285F97385FA747E017F00E57412B6
:103A99006595E5732FFF50010E8E5A8F5B900013C9
:103AA900E0FCA3E0FDEF2DFDEE3CFC8C5C8D5D227E
:103AB90075A71085F97385FA747E017F00E5741284
:103AC9006595E5732FFF50010E8E5A8F5B9000DCD0
:103AD900E0B40210AC2CAD2DEF2DFDEE3CFC8C5C5E
:103AE9008D5D8016AE5AAF5B900013E0FCA3E0FD3C
:103AF900EF2DFDEE3CFC8C5C8D5D22AE5AAF5B7404
:103B09000A8E048F05FF1265858C5C8D5DAE5AAFF8
:103B19005B740A8E048F05FF1265B08C5A8D5BE5C4
:103B29005B455A6013740AC3955BFFE4955AFE8E90
:103B39005A8F5B785C1265E9E573A85CB80015D308
:103B4900955D4010E573C3955DFFE4955CFE8E5C61
:103B59008F5D8010E5732424C3955DFFE4955CFEB9
:103B69008E5C8F5DAE5CAF5D74246F4E700B755DBE
:103B790023755C0075730180037573002290008AB8
:103B8900E0B40104C2108002D21090008BE0B401AD
:103B990004C2118002D2119000C8E075F0DCA4FFC4
:103BA900AEF0740A8E048F05FF1265859007B0EC9C
:103BB900F0A3EDF0A20D401674038C068D07126573
:103BC9009574011200399007AEEEF0A3EFF07E0173
:103BD9007F00900086E01265959000C9E08E048F01
:103BE90005FF126585740AFF1265858D609000D204
:103BF900E075F0DCA4FFAEF0740A8E048F05FF12A5
:103C090065859007B4ECF0A3EDF09000D4E0601363
:103C19009000D4E0F5F0741684FF7E00EF9007C29F
:103C2900F0800674649007C2F09000CAE090006EBC
:103C3900F0900114E0900058F09000A3E090005A31
:103C4900F09000CCE090005BF0900078E090005C90
:103C5900F09000FEE0900061F0900162E090006257
:103C6900F0900163E0900063F0900164E0900064DB
:103C7900F0A227B34016900162E0700C900163E056
:103C89007006900164E060028002C22774E390002C
:103C99006DF09000B3E0B40B0874E390006DF08010
:103CA9005A9000B3E0B419129000C9E09063EA1287
:103CB900008CE49390006DF080419000B3E0B41E55
:103CC900129000C9E090640812008CE49390006D92
:103CD900F080289000B3E0B428129000C9E0906405
:103CE9003212008CE49390006DF0800F9000B3E0E5
:103CF900B446089000AAE090006DF09000E3E0FE61
:103D09009000B1E06E600A9000B1E09000E3F0D25B
:103D190026900071E0FE9000B0E0B5063390007384
:103D2900E0FE9000CEE0B50627900072E0FE90001C
:103D3900DCE0B5061B900075E0FE900083E0B50657
:103D49000F900074E0FE9000BEE06E7003023E9991
:103D5900900049E0C39405500874029000FFF08078
:103D6900149000DCE0600874089000FFF08006748D
:103D79000A9000FFF0900083E0B4010674009000FF
:103D8900E9F0900083E0B4020674009000CEF09050
:103D99000083E0B4030674009000DBF09000CEE0ED
:103DA900D3940140147418900101F074009006C86E
:103DB900F074009006C9F0800C7400900101F07451
:103DC900189006C8F09000B0E06014741A9000973B
:103DD900F074009006D0F074009006D1F0800C7455
:103DE90000900097F0741A9006D0F09000B0E0B4FB
:103DF90002147419900098F074009006CCF07400C5
:103E09009006CDF0800C7400900098F0741990061B
:103E1900CCF09000DCE0700E74059006DCF07406BE
:103E29009006E0F0801874009006DCF074009006AB
:103E3900DDF074009006E0F074009006E1F0D226FF
:103E49009000B0E0900071F09000DCE0900072F01A
:103E59009000CEE0900073F09000BEE0900074F006
:103E6900900083E0900075F0900083E0900059F095
:103E79009000BEE090005DF09000DCE090005EF004
:103E89009000B0E090005FF09000CEE0900060F00C
:103E99009000E6E0B4011790001F740FF0A374FFBF
:103EA900F0900021E4F0A3F074029000E6F0900095
:103EB900E6E0B40341900021E0FEA3E0FF90001F7B
:103EC900E0FCA3E0FD1265E1741012659574081217
:103ED9000039EF90006AF0EF700674FF90006AF005
:103EE90074009000E6F0900020E090006BF09000E4
:103EF9001FE090006CF0900077E090003BF090009C
:103F09003BE0241290003CF090003CE0D394244024
:103F19000B90003CE0C3942490003CF090003FE4F7
:103F2900F090003BE0B4240C90003F7401F0900045
:103F39003B7401F0900040E4F090003CE0B4240CA4
:103F49009000407401F090003C7401F0900077E01B
:103F5900FE9000DAE02E900042F0900042E06412F8
:103F69006007900042E0B42406900042E004F0901B
:103F79000042E0D39424400B900042E0C394249083
:103F89000042F0900042E0D39412400D900042E0CC
:103F9900C39412900043F0800A900042E0241290EA
:103FA9000043F07551129000BDE090003DF0900083
:103FB9003DE075F01284AFF07E00EF4E7006900080
:103FC9003DE004F090003DE0B4490690003D7401E5
:103FD900F090003DE0D39424400F90003DE0C3945D
:103FE9002490003DF0D2208002C22090003DE0D311
:103FF9009412400D90003DE0C3941290003EF08071
:104009000A90003DE0241290003EF022C293C2942F
:10401900C291C292C287C290E5B554EFF5B5E5B534
:1040290054DFF5B5C296C295C2A0C297C2A2C2A179
:10403900E5B554BFF5B5E5B5547FF5B5E5B554FB20
:10404900F5B5C212755E469000C0E07005756D0247
:104059008003756D0375550075540090000874FF51
:10406900F0A374DCF0C217C21974C8900033F0745D
:10407900C8900037F0755300755200C20D7546009F
:10408900E56FB40903756F00756300900015E4F0DE
:10409900A3F0757010C215C2169007B0E0FEA3E038
:1040A900FF740312659574011200399007AEEEF0A2
:1040B900A3EFF0C20275570075560090000CE4F0AA
:1040C900A3F0C228755900755800900082E075F078
:1040D90032A4FDACF090001DECF0A3EDF0C238A2C3
:1040E9002CB39205A22DB39206A22EB39207A22F4A
:1040F900B39208A230B39209A231B3920AA232B3A1
:10410900920BA233B3920C2285F97385FA747E015E
:104119007F00E574126595E5732FFF50010E8E5AE5
:104129008F5BAC5CAD5DEF2DFDEE3CFC8C5C8D5D79
:10413900D293D294E55DF5FBE55CF5FCE55DF5E927
:10414900E55CF5EA9000BEE0B40314D291D292E5A1
:104159005DF5EBE55CF5ECE55DF5EDE55CF5EE228D
:1041690075A71085F97385FA747E017F00E57412CD
:104179006595E5732FFF50010E8E5A8F5B7E017F87
:10418900769000FBE0126595AC5AAD5BED2FFFEC24
:104199003EFE8E5C8F5DE55DF5FDE55CF5FE90000C
:1041A9006EE4F075A7007412900045F02285F9734A
:1041B90085FA747E017F00E574126595E5732FFF1A
:1041C90050010E8E5A8F5B9007B0E0FCA3E0FDEF23
:1041D9002DFDEE3CFC8C5C8D5DE55DF5FDE55CF54A
:1041E900FE220564229000BEE0B403539000DCE097
:1041F900B4012EA2D8B34004C293C287A2D9B34056
:1042090004C294C290A2DAB34008C291E5B554EF52
:10421900F5B5A2DBB34008C292E5B554DFF5B58028
:104229001CA2D8B34002C293A2D9B34002C294A23D
:10423900DAB34002C291A2DBB34002C292801EA24D
:10424900D8B3400AC2939000DCE06002C287A2D9C9
:10425900B3400AC2949000DCE06002C290A2DCB3D1
:104269004004C296C29575D8402285A77275A710D9
:10427900A2D8B34002C287A2D9B34002C290A2DA3F
:10428900B34006E5B554EFF5B5A2DBB34006E5B595
:1042990054DFF5B5A2DCB340089000CAE090006E87
:1042A900F075D8408572A722900047E493640660B0
:1042B9000280FE74C89007B6F8E4F0E8A3F075B57B
:1042C9000075840175A70075FFA0900041E4F075A1
:1042D900C91075A70F75A1C775A70075D90075CE47
:1042E9000C75A70F75F1FE75F2FF75F30775F47874
:1042F90075A4BA75A5FF75A60775AE0075AFFF75EC
:10430900D48175D5FF75D6FF75D7FF75A70075A23E
:104319000175A14775F80975D80075D90475DA09C9
:1043290075DB0975DC0975DD0975DE0975D8407518
:10433900A71075D80075D90475DA0975DB0975DC1C
:104349000975DD0975DE0975D84075A70075E60898
:1043590075E71075BC0175BE0475BD6C75BE077532
:10436900BDA075BE0875BD0175BC0075BB1875BCCF
:104379002075BA0875E88075D11375A70F75E10521
:1043890075E20075C74012401575970075978074DE
:104399000A1265757597C0E5975420700280F87503
:1043A9008F0275A700D2AF75980075A90C75A70F74
:1043B90075AB4375ADFB75AC1E75A71075C918753E
:1043C900CA0075CB0075C80475A700758912758E6A
:1043D90004758C00758A00C2A9D28C758D00758B05
:1043E90000D2ABD28E75EF0675D944C29974C8F55F
:1043F900097508001200E975B5001204E9746390A3
:1044090007B6F8E4F0E8A3F012037574C89007B68C
:10441900F8E4F0E8A3F07464F5097508001200E9FE
:10442900900059E0900083F0900083E0D39403401A
:104439000C7400900083F07400900059F0C21D9034
:104449000083E0905DDDF82828738028A2B440023B
:10445900D21D802075A70F75F30F75A700A2A34081
:1044690002D21D800F75A70F75F31775A700A2A4B7
:044479004002D21D0E
:0C5DDD0002445302445502445D02446E2F
:10447D00A21DB3405F757308E573D3940E5020E50C
:10448D00739007B6F8E4F0E8A3F01202447464F5F3
:10449D00097508001200E97873740126F650D97475
:1044AD00029000BFF0900059E0900083F0900083DF
:1044BD00E0905DE9F8282873801674009000E9F00B
:1044CD00800E74009000CEF0800674009000DBF03A
:0C5DE9000244C50244C70244CF0244D764
:1044DD00D21C805D757301E573D394075020E5738D
:1044ED009007B6F8E4F0E8A3F01202447464F509FD
:1044FD007508001200E97873740126F650D974011D
:10450D009000BFF0900059E0900083F0900083E0A0
:10451D00905DF5F8282873801674009000E9F080FE
:0F452D000E74009000CEF0800674009000DBF05A
:0C5DF50002452402452602452E024536D8
:10453C00C21C900058E0900114F0900059E09000DB
:10454C0083F090005AE09000A3F090005BE09000A4
:10455C00CCF090005CE0900078F090005DE0900072
:10456C00BEF090005EE09000DCF090005FE0900008
:10457C00B0F0900060E09000CEF0900061E0900010
:10458C00FEF0900062E0900162F0900063E0900118
:10459C0063F0900064E0900164F0900162E0700CB4
:1045AC00900163E07006900164E060028004C22711
:1045BC008002D2279000C9E07006740A9000C9F0FE
:1045CC009000AAE0700674E39000AAF09000B0E0AE
:1045DC0004900071F09000B1E09000E3F0123B8683
:1045EC00E5B54401F5B57406900047F074019000F0
:1045FC0048F0740390004AF0740590004BF0740E70
:10460C0090004CF0740590004DF0900049E0B4041B
:10461C0006740490004DF0740190004EF0740090FC
:10462C000053F07400900056F074FF900057F07433
:10463C003390014DF0743690014EF0742D90014F73
:10464C00F07431900150F07420900151F07434905A
:10465C000152F07443900153F07479900154F0744A
:10466C006C900155F07420900156F0742090015715
:10467C00F07420900158F07420900159F07420903F
:10468C00015AF0742090015BF09000E5E090006A14
:10469C00F090009CE090006BF090009DE090006C1E
:1046AC00F0A2B6B3920EA2B3B3920FA2A4B392230C
:1046BC00A2B4B39224A2A3B39225900066E4F07541
:1046CC006F00743A900776F074FD900777F09000C5
:1046DC0067E4F09007B0E0FEA3E0FF740312659569
:1046EC0074011200399007AEEEF0A3EFF0756E0175
:1046FC00900045E4F0C222756300C213D214C202CA
:10470C00757100C22AD203C22BD204C22CD205C2AC
:10471C002DD206C22ED207C22FD208C230D209C265
:10472C0031D20AC232D20BC233D20CC21EC21FC249
:10473C0020C221C22612009E755F00756B00756148
:10474C0000756532756600756700756800756900DF
:10475C00756A00900015E4F0A3F0756C00D2B2D22B
:10476C00A4D2B0D2B1D2A3D2A7D2A6D2A5D2B7909E
:10477C000082E0D394FA400674FA900082F07E0135
:10478C007F0090006CE012659590006BE02FFF505D
:10479C00010E90001FEEF0A3EFF0EFD394FFEE9418
:1047AC000F400790001FE4F0A3F090006AE0700641
:1047BC0074FF90006AF09000BFE0D394024006743E
:1047CC00019000BFF09000C0E07005756D02800391
:1047DC00756D039000C1E0D3940140067400900005
:1047EC00C1F09000C7E0C3940A5006740A9000C749
:1047FC00F09000D1E0700674019000D1F09000D1DF
:10480C00E0B4FF0674FE9000D1F09000D8E0D39491
:10481C00FE400674FE9000D8F09000FEE0D39402A7
:10482C00400674019000FEF0900114E0D394014016
:10483C00067401900114F074019000DEF074019084
:10484C0000DFF074009000E6F07400900102F07448
:10485C0000900106F074299006BCF0742A9006C0F2
:10486C00F074179006C4F0741B9006D4F0741C906E
:10487C0006D8F0D29C9000B1E0D3940440067404A6
:10488C009000B1F0E570D394104003757010900651
:10489C00BDE0D3940C400674009006BDF09006C1A8
:1048AC00E0D3940C400674009006C1F09006C5E06D
:1048BC00D3940C400674009006C5F09006C9E0D362
:1048CC00940C400674009006C9F09006CDE0D39489
:1048DC000C400674009006CDF09006D1E0D3940CF9
:1048EC00400674009006D1F09006D5E0D3940C40AD
:1048FC000674009006D5F09006D9E0D3940C4006CF
:10490C0074009006D9F09006DDE0D3940C40067448
:10491C00009006DDF09006E1E0D3940C40067400A4
:10492C009006E1F0D2EC75CF01A298B34005C29885
:10493C00120646E54D6006A299B3B340028005C24B
:10494C0099120C57E54E64016005E54EB4040280E3
:10495C00D5C28E7E107F00E564126595E58D75F0ED
:10496C0010A4FDACF0EF2DFDEE3CFCE58B75F010CA
:10497C0084FF7E00ED2FFFEC3EFE8E548F55D28EC1
:10498C009000A3E060099000A3E0C3943D40028036
:10499C005C9000171265A3900017E0FEA3E0FF9057
:1049AC000019E0FCA3E0FDEFB50542EEB5043EB204
:1049BC001BA20DB3401975E700A21BB34008E5B567
:1049CC004404F5B58006E5B554FBF5B575E71090D4
:1049DC000019E0FEA3E0FF90001BE0FCA3E0FDEF5C
:1049EC002DFDEE3CFC900019ECF0A3EDF09000B026
:1049FC00E060099000B0E0C394034002806F122D78
:104A0C0096A20DB35009900066E0C3942B4002802F
:104A1C000690009AE0F545E54575F005A4FFAEF06B
:104A2C009007B8EEF0A3EFF0900087E0C3956140DB
:104A3C0007E55FC3956050079007B8E4F0A3F0AEAC
:104A4C002EAF2F9007B8E0FCA3E0FDEFD39DEE9CBA
:104A5C004004C2A1800B900066E0C394415002D286
:104A6C00A19000B0E0B40205A2A1B392A29000B054
:104A7C00E0B4031C122EB1AE2EAF2F9007B8E0FCA1
:104A8C00A3E0FDEFD39DEE9C4004D2A18002C2A115
:104A9C0090008BE06009A2B3300F01B3B3400280E9
:104AAC0039A2B3300F01B34031A2B3301101B3407E
:104ABC001C9000BEE0B40306A21EB3B340028006F5
:104ACC007404900045F0D21EA211B3920FA211B340
:104ADC0030B301B34004A211920FA2B6300E01B351
:104AEC00500302516AA2B6300E01B3500302516A50
:104AFC00A2B6301001B35003024F8E756E009000B9
:104B0C00A3E0B43D1975E700A210B34008E5B55415
:104B1C00FBF5B58006E5B54404F5B575E710055E03
:104B2C00A212B3B35013AE54AF55900008E0FCA3DF
:104B3C00E0FDEDC39FEC9E4003024C8EE56DB4038B
:104B4C002EA228B34022E55EB42403756D01E55E08
:104B5C00C3942450069000457401F0E55ED3942470
:104B6C0040067402900045F0755E01D228805AE52B
:104B7C006DB40206756D01755E24E55EB424057591
:104B8C005E018045900045E07030E55EC394245092
:104B9C00069000457401F0E55ED39424400674023F
:104BAC00900045F0E55EC394245002D222E55ED31A
:104BBC0094244002D222C296C2959000C0E0B40167
:104BCC00051240158003755E01AE56AF57AC54AD5F
:104BDC0055EF2DFDEE3CFC7403FF1265858C568D54
:104BEC00579000A3E060099000A3E0C3943D4002FD
:104BFC008043900017E0FEA3E0FF9000A3E08E043A
:104C0C008F05FF12658574018C068D071200399093
:104C1C00001BEEF0A3EFF090001BE0F8A3E0900077
:104C2C0019C8F0A3C8F0900017E4F0A3F0C21BE57C
:104C3C00B554FBF5B5A2B4B34002C224A2A4B34050
:104C4C0002C223A2A3B34002C225A222B34002C2D5
:104C5C0022A21EB34006A220921F8002B21F900017
:104C6C008BE06012E56D700EA21EB35009A21F30CE
:104C7C002001B3B3400280067405900045F0C21EBB
:104C8C00803AAE56AF57AC54AD55EF2DFDEE3CFC13
:104C9C0074018C068D071200398E568F57E56DC343
:104CAC009402500DAC54AD557488C39D74139C4044
:104CBC000280091240157406900045F0E55EB4249C
:104CCC00127403900045F0D2229000C0E0B40103AE
:104CDC00124015AE58AF59AC54AD55EF2DFDEE3C0E
:104CEC00FC8C588D59AE54AF55EFD39DEE9C4011B2
:104CFC0090000FE0FAA3E0FBEBC394E8EA940340C6
:104D0C0002800690000F1265A390000CE0FEA3E059
:104D1C00FFAC54AD55EF2DFDEE3CFC90000CECF0CF
:104D2C00A3EDF09000C0E0B4011DAE54AF55740576
:104D3C0012659574038E048F05FF1265859000082B
:104D4C00ECF0A3EDF08016AE54AF557403126595DC
:104D5C007401120039900008EEF0A3EFF0C28E75CA
:104D6C008D00758B00756400755501755400D28EDD
:104D7C00E55E240875F00984AFF07E00EF4E707587
:104D8C0090000CE0F8A3E090000AC8F0A3C8F090E3
:104D9C00000AE0FEA3E0FFEF4E600B7C7B7D8912E6
:104DAC0064838E528F5390000CE4F0A3F0AE52AF9C
:104DBC00537428BE00039F5010E5632FFF50010E63
:104DCC0074011200398E528F538553639000C7E0E3
:104DDC00A852B8000DD395534008E553900044F009
:104DEC0080099000C7E014900044F0E56D600675F2
:104DFC0053007552009000BEE0B4030890003DE0F3
:104E0C00655E6002800BA21FB34004D2218002B207
:104E1C0021E55E640B6005E55EB41D099000B0E011
:104E2C0060031223D2900042E0655E60079000435D
:104E3C00E0B55E03756F00A213B35006A212B3B3B4
:104E4C004003024EF690007CE0B401739000FEE04B
:104E5C00B40214120E2690006FE075F0BEA4FFAEE3
:104E6C00F08E5C8F5D8056E56775F00A84FF7E00DE
:104E7C009005761265BCE0F55B755A00AE5AAF5BD7
:104E8C009000A1E012659574648E048F05FF126585
:104E9C00858C5C8D5DE55D90000EF0AE5AAF5B903D
:104EAC00007AE012659574648E048F05FF12658597
:104EBC0074BE8C068D071265958E5C8F5D80179085
:104ECC00007AE075F0BEA4FFAEF08E5C8F5D9000B2
:104EDC00A1E090000EF0E561C394CC5006E55D4571
:104EEC005C70028003124111D213E56DB40106E52A
:104EFC005E640B600280097570019000467401F0CD
:104F0C00E56D70799000C3E0600D90006EE0A852E2
:104F1C00B800069553400280389000C3E0B40217E5
:104F2C0090003BE0655E600790003CE0B55E037569
:104F3C007003756C00800CC200756C00900015E459
:104F4C00F0A3F090006EE060067409900045F080CC
:104F5C002C90003BE0655E600790003CE0B55E0382
:104F6C0075700190003BE0B55E069000467401F050
:104F7C0090003CE0B55E067402900046F0A210B3BF
:104F8C00920EA210B330B601B3500302516A756E83
:104F9C00019000A3E0B43D1975E700A210B34008DE
:104FAC00E5B54404F5B58006E5B554FBF5B575E7F4
:104FBC0010E5B54401F5B5742B900066F0A2109283
:104FCC000EE55ED3944A4014D212E55ED3946E4043
:104FDC000B7404900045F0D222755E469000CBE035
:104FEC00B40107E56AC39414400280091240157499
:104FFC0013900045F0A22A300301B3501D75E70051
:10500C00A22AB34008E5B54408F5B58006E5B554C9
:10501C00F7F5B575E710A22A9203A22B300401B361
:10502C00501D75E700A22BB34008E5B54402F5B559
:10503C008006E5B554FDF5B575E710A22B9204A2D8
:10504C002C300501B3500FA22CB34004D2A0800227
:10505C00C2A0A22C9205A22D300601B3500FA22D96
:10506C00B34004D2978002C297A22D9206A22E3092
:10507C000701B3500FA22EB34004D2A28002C2A2E9
:10508C00A22E9207A22F300801B3500FA22FB340CB
:10509C0004D2A18002C2A1A22F9208A23030090131
:1050AC00B3501D75E700A230B34008E5B54440F598
:1050BC00B58006E5B554BFF5B575E710A230920979
:1050CC00A231300A01B3501D75E700A231B340087C
:1050DC00E5B54480F5B58006E5B5547FF5B575E7C3
:1050EC0010A231920AA232300B01B3500FA232B38C
:1050FC004004D2878002C287A232920BA233300CBA
:10510C0001B3500FA233B34004D2908002C290A2DC
:10511C0033920CE56AC394415009740E900045F02B
:10512C0012401590004DE0FE900049E004C39E40F3
:10513C0009900049E0D39408400974FB900045F0B5
:10514C00124015900052E06015900052E0FE900065
:10515C004CE06E600974FE900045F0124015A222DE
:10516C00B34004C296C2959000FBE0600CAE52AF07
:10517C00537414BE00059F40028048900083E09059
:10518C005E01F8282873803BA2B4B35005A224B367
:10519C0040028005124169D2248028A2A3B3500595
:1051AC00A225B340028005124169D2258015A2A424
:1051BC00B35005A223B340028005124169D223806B
:0351CC000280005E
:105E01000251920251940251A70251BA0251CD029C
:025E110051CF6F
:1051CF00A215B3B3500890003DE0655E6003025234
:1051DF00AEA201B35006A200B3B340030252AA908D
:1051EF0000BEE0B40302800302527FA20DB34067FA
:1051FF00A221B3402D123A8CE55DF5FBE55CF5FC81
:10520F00D293A202B34002D2879000DCE0B4021026
:10521F00123AB9E55DF5FBE55CF5FC75A700D287A1
:10522F008033123A8CE55DF5EBE55CF5ECD291A29B
:10523F0002B34006E5B54410F5B59000DCE0B402CA
:10524F0014123AB9E55DF5EBE55CF5EC75A700E5F1
:10525F00B54410F5B58017123A8CE55DF5FBE55CAA
:10526F00F5FCE55DF5EBE55CF5ECD293D291802B87
:10527F00123A8CE55DF5FBE55CF5FCD293A202B327
:10528F004002D2879000DCE0B40210123AB9E55D1B
:10529F00F5FBE55CF5FC75A700D287C215D216A207
:1052AF0016B3B3500890003EE0655E600302538D65
:1052BF00A201B35006A200B3B3400302538990007A
:1052CF00BEE0B40302800302535EA20DB34067A297
:1052DF0021B3402D123A8CE55DF5E9E55CF5EAD294
:1052EF0094A202B34002D2909000DCE0B4021012FC
:1052FF003AB9E55DF5E9E55CF5EA75A700D290806E
:10530F0033123A8CE55DF5EDE55CF5EED292A20233
:10531F00B34006E5B54420F5B59000DCE0B40214C7
:10532F00123AB9E55DF5EDE55CF5EE75A700E5B56B
:10533F004420F5B58017123A8CE55DF5E9E55CF58B
:10534F00EAE55DF5EDE55CF5EED294D292802B1295
:10535F003A8CE55DF5E9E55CF5EAD294A202B3403B
:10536F0002D2909000DCE0B40210123AB9E55DF57C
:10537F00E9E55CF5EA75A700D290D215C216E57083
:0E538F00905E13F82828730257C29000B1E018
:065E1300025396025399B0
:10539D00905E46F8282873121EAE8012121EAE8043
:0E53AD000D121F388008121FE48003121FE447
:0F5E46000253A40253A90253AE0253B30253B83E
:1053BB007570020257C2122110122227A238B34075
:1053CB00229000A5E0F56C900076E0256CFE900035
:1053DB0044E075F01E84FC7F00EE2CF536741090C3
:1053EB000045F09007AEE0FEA3E0FF740A1265954E
:1053FB0090000AE0FCA3E0FD74098F02FF126585A3
:10540B008D078C038E048A058B061264839007B27A
:10541B00EEF0A3EFF09000CCE0B401087478BE007E
:10542B00059F4002800D74789007B2F8E4F0E8A372
:10543B00F0801B9007B2E0FEA3E0FF74F0BE000308
:10544B009F500B74F09007B2F8E4F0E8A3F0E53648
:10545B0070037536019007B2E0FEA3E0FFE5362F2F
:10546B00FF50010E9007B2EEF0A3EFF075700390B2
:03547B000046E008
:035E19000253C170
:10547E00905E55F82828738010A239400375700A83
:09548E008007A239400375700B80
:095E5500025485025487025490A6
:105497000257C29006BDE060031224EA9000FCE0C8
:1054A700B401149000FDE0A852B8000495535007CA
:1054B700E55FC39560400280097415900045F002CE
:1054C700554A9000B1E0D39402403F900085E02414
:1054D70003A852B8000495535009900087E0D3956C
:1054E7006150028008D2017408900045F090008551
:1054F700E0A852B80005D39553500B900087E024DD
:1055070003C395615002C2018039900085E02403EE
:10551700A852B8000495535007E55FC39560400251
:105527008008D2017408900045F0900085E0A852E9
:10553700B80005D395535009E560240FC3955F5014
:1055470002C2019000CBE07007E56AC394144002E1
:105557008002D201A2014005757004800A7570109F
:10556700900015E4F0A3F0A20DB34029E56775F0AC
:105577000A84FF7E009005761265BCE0C3946950EB
:1055870005122407800F9007B0E0F8A3E09007AE5C
:0C559700C8F0A3C8F00257C29000B1E0B9
:065E1C0002549A02559F9A
:1055A300905E5EF8282873120F108012120F10807D
:0E55B3000D1210BE80081211708003121170CC
:0F5E5E000255AA0255AF0255B40255B90255BEFE
:1055C1009006C1E060031225C67570050257C2122C
:1055D10012B07570069006C5E060031226B69006FB
:1055E100C9E060031227920257C290000EE06006E4
:1055F100A20DB3B34002801D90000EE02529FFAE3D
:105601002850010E8E288F29E55ED3941250069002
:10561100000EE014F01214F67570079006CDE060EC
:105621000312286E9006D1E0600312294A0257C284
:105631009000FEE0B40203120E9E1218F575700878
:105641009006D5E06003122A269006D9E060031285
:105651002B020257C2121CB1A215B35005A216B3F8
:1056610040028004D215D2167570109006DDE060FC
:1056710003122BDE9006E1E06003122CBA0257C23E
:105681000257C2900035E0C394465008C296744652
:10569100900035F090003FE0B4011DE536240AF595
:1056A100369007B2E0FEA3E0FF740A2FFF50010E0F
:1056B1009007B2EEF0A3EFF085365B755A009000CB
:1056C1003BE0F573123B04E55D900035F09000047A
:1056D100E55AF0A3E55BF0E573900036F0C218904F
:1056E10007B2E0F55AA3E0F55B90003BE0F57312D9
:1056F1003B04E55D900033F0900000E55AF0A3E52E
:105701005BF0E573900034F0C217E56DB4010575E7
:10571100700B80037570030257C2900039E0C39487
:105721004650139000CCE0B40104C2968002C295A9
:105731007446900039F0900040E0B4011DE5362434
:105741000AF5369007B2E0FEA3E0FF740A2FFF507E
:10575100010E9007B2EEF0A3EFF085365B755A00AB
:1057610090003CE0F573123B04E55D900039F09048
:105771000006E55AF0A3E55BF0E57390003AF0C24C
:105781001A9007B2E0F55AA3E0F55B90003CE0F512
:1057910073123B04E55D900037F0900002E55AF08A
:1057A100A3E55BF0E573900038F0C219E56DB40133
:1057B10003756D0075700380088006800480028087
:0157C10000E7
:105E22000255D00255EB02563102565602568102F5
:105E3200568402571B0257BA0257BC0257BE02577A
:045E4200C00257C281
:1057C200900033E0B55E73A217404F900000E0FEF8
:1057D200A3E0FFEF4E6021AE56AF57900000E0FC11
:1057E200A3E0FD120003740A8E048F05FF12658583
:1057F200900000ECF0A3EDF0900034E0601A90000D
:1058020000E0FEA3E0FFAC56AD57EF2DFDEE3CFCF1
:10581200900000ECF0A3EDF0D217AE54AF5590001B
:1058220000E0FCA3E0FDEFC39DEE9C400D1241B6EB
:10583200D296C21774C8900033F0A217B3B35007C0
:10584200900033E0B55E02800D1241B6D29674C864
:10585200900033F0C217900035E0B55E70A2184098
:105862004F900004E0FEA3E0FFEF4E6021AE56AF82
:1058720057900004E0FCA3E0FD120003740A8E04BA
:105882008F05FF126585900004ECF0A3EDF0900007
:1058920036E0601A900004E0FEA3E0FFAC56AD577C
:1058A200EF2DFDEE3CFC900004ECF0A3EDF0D218DD
:1058B200AE54AF55900004E0FCA3E0FDEFC39DEEB3
:1058C2009C400AC2967446900035F0C218A218B3E2
:1058D200B35007900035E0B55E02800AC296744666
:1058E200900035F0C218900037E0B55E7EA21940F4
:1058F2004F900002E0FEA3E0FFEF4E6021AE56AFF4
:1059020057900002E0FCA3E0FD120003740A8E042B
:105912008F05FF126585900002ECF0A3EDF0900078
:1059220038E0601A900002E0FEA3E0FFAC56AD57EB
:10593200EF2DFDEE3CFC900002ECF0A3EDF0D2194D
:10594200AE54AF55900002E0FCA3E0FDEFC39DEE24
:105952009C40181241B69000CCE0B40104D296806B
:1059620002D295C21974C8900037F0A219B3B3508D
:1059720007900037E0B55E0280181241B69000CC65
:10598200E0B40104D2968002D29574C8900037F038
:10599200C219900039E0B55E7BA21A404F90000612
:1059A200E0FEA3E0FFEF4E6021AE56AF5790000637
:1059B200E0FCA3E0FD120003740A8E048F05FF12BF
:1059C2006585900006ECF0A3EDF090003AE0601AD5
:1059D200900006E0FEA3E0FFAC56AD57EF2DFDEEC2
:1059E2003CFC900006ECF0A3EDF0D21AAE54AF5599
:1059F200900006E0FCA3E0FDEFC39DEE9C401590F5
:105A020000CCE0B40104C2968002C29574469000B4
:105A120039F0C21AA21AB3B35007900039E0B55E4A
:105A22000280159000CCE0B40104C2968002C295B7
:105A32007446900039F0C21A9000CEE0B40202809F
:105A420003025B56900068E0D3956650649000684C
:105A5200E0F4042566FE9000D1E08E00F5F0E884C3
:105A6200FF7E008F73EFC39410500CEF8573F0A488
:105A7200FDACF08D7380037573FF900068E0D395E1
:105A820073400B900068E0C39573F57180037571E4
:105A9200009000ECE0D3957140069000ECE0F571C7
:105AA2009000EDE0C3957150069000EDE0F5718035
:105AB20071900068E0C39566FE9000D1E08E00F51B
:105AC200F0E884FF7E008F73EFC39410500CEF85D3
:105AD20073F0A4FDACF08D7380037573FF85735B67
:105AE200755A00900068E0255BFFAE5A50010E8E99
:105AF2005A8F5B74FFBE0009D39F4005855B71809E
:105B0200037571FF9000ECE0D3957140069000ECB4
:105B1200E0F5719000EDE0C3957150069000EDE064
:105B2200F571A20DB3B3500D900069E0FE9000D95B
:105B3200E0D39E5002800A7407900045F0C297801D
:105B42001375A710E5CDC395714004C2978002D2A8
:105B52009775A700E56FC39409500AA2EDB34005FB
:105B6200C2ED123050AE54AF557410C39F74279ECD
:105B7200400C900067E0C3945A4003025DDAA2121F
:105B8200B340091240157406900045F0A21DB340BF
:105B920008E5B54404F5B58006E5B554FBF5B5A2B4
:105BA20014B3500EE561D394334007E561C394CC3E
:105BB200400280419000FEE0B40214120E269000D2
:105BC2006FE075F050A4FFAEF08E5C8F5D800F9099
:105BD200007AE075F050A4FFAEF08E5C8F5DE55D5B
:105BE200455C6011E5B54401F5B5742B900066F093
:105BF200124111D214900067E0D394014007E5618D
:105C0200C3941A40028002C2149006BDE0600312DF
:105C120024EAA22A300301B35017A22AB34008E5AE
:105C2200B54408F5B58006E5B554F7F5B5A22A9254
:105C3200039006C1E060031225C6A22B300401B313
:105C42005017A22BB34008E5B54402F5B58006E52E
:105C5200B554FDF5B5A22B92049006C5E06003127F
:105C620026B6A22C300501B3500FA22CB34004D2A9
:105C7200A08002C2A0A22C92059006C9E060031285
:105C82002792A22D300601B3500FA22DB34004D2A9
:105C9200978002C297A22D92069006CDE060031271
:105CA200286EA22E300701B3500FA22EB34004D2A9
:105CB200A28002C2A2A22E92079006D1E060031235
:105CC200294AA22F300801B3500FA22FB34004D2A9
:105CD200A18002C2A1A22F92089006D5E060031211
:105CE2002A26A230300901B35017A230B34008E58A
:105CF200B54440F5B58006E5B554BFF5B5A230927E
:105D0200099006D9E06003122B02A231300A01B3D6
:105D12005017A231B34008E5B54480F5B58006E5D9
:105D2200B5547FF5B5A231920A9006DDE060031208
:105D32002BDEA232300B01B3500FA232B34004D299
:105D4200878002C287A232920B9006E1E0600312C2
:105D52002CBAA233300C01B3500FA233B34004D299
:105D6200908002C290A233920C900067E0C3945AD2
:105D72005010E56FB40909900067E004F0756F00F8
:105D8200803BE56FB40903756F00755500755400CB
:105D9200758D00758B00756400900066E0C39441B8
:105DA2005008900066E004F080067441900066F0AE
:105DB200900066E0B44106E5B554FEF5B590006783
:105DC200E0D394014007E56AC3944140028009741C
:0B5DD2000E900045F01240150249320F
:105E6D000000010001400160018001A001C001E0BE
:105E7D0002000300039603B603D603F404000500E5
:105E8D000512052405360548055A056C057E059055
:105E9D0005A805C005DE0600061406280646066E92
:105EAD0006AE05CF00FF013F015F017F019F01BFDE
:105EBD0001DF01FF02FF039503B503D503F303FFD4
:105ECD0004FF05110523053505470559056B057DAE
:105EDD00058F05A705BF05CE05F106130627064557
:105EED00066D06AD06ED05DD0FAA0FA50F9F0F9AE6
:105EFD000F940F8D0F870F800F780F710F680F6044
:105F0D000F570F4E0F450F3B0F300F250F1A0F0E6A
:105F1D000F020EF50EE80EDB0ECC0EBE0EAE0E9F72
:105F2D000E8E0E7D0E6C0E5A0E470E340E200E0C7C
:105F3D000DF70DE20DCB0DB50D9D0D850D6D0D54B0
:105F4D000D3A0D200D050CE90CCE0CB10C940C7610
:105F5D000C580C3A0C1B0BFB0BDB0BBB0B9A0B7988
:105F6D000B570B350B130AF10ACE0AAB0A870A64DD
:105F7D000A400A1C09F809D409B0098C09670943BC
:105F8D00091F08FB08D608B2088E086A08460823C0
:105F9D0007FF07DC07B9079607730751072F070D92
:105FAD0006EC06CA06AA068906690649062A060AE5
:105FBD0005EC05CD05B0059205750558053C052088
:105FCD00050504EA04CF04B5049C04820469045158
:105FDD0004390422040B03F403DE03C803B2039D4A
:105FED00038903750361034D033B03280316030463
:105FFD0002F202E102D102C002B002A002910282BD
:10600D000273026502570249023C022F0222021658
:10601D00020901FD01F201E601DB01D001C601BB60
:10602D0001B101A7019D0194018B018201790170DC
:10603D0001680160015801500148014101390132E7
:10604D00012B0125011E01180111010B010500FF96
:10605D0000FA0FA60FA00F990F920F8B0F840F7CD4
:10606D000F740F6B0F620F580F4E0F430F380F2C1D
:10607D000F1F0F120F050EF70EE80ED80EC80EB734
:10608D000EA50E930E800E6C0E580E420E2C0E1594
:10609D000DFD0DE40DCB0DB10D950D790D5D0D3F84
:1060AD000D200D010CE10CC00C9E0C7C0C590C3517
:1060BD000C100BEA0BC40B9E0B760B4F0B260AFD37
:1060CD000AD40AAA0A800A550A2A09FF09D409A87E
:1060DD00097C0950092508F908CD08A10875084A59
:1060ED00081E07F307C8079D07730749072006F722
:1060FD0006CE06A6067E06570630060A05E405BF3F
:10610D00059B057705540532051004EF04CE04AE4A
:10611D00048F047104530435041903FD03E203C70E
:10612D0003AD0394037B0363034B0334031E030886
:10613D0002F302DE02CA02B602A30291027F026DD1
:10614D00025C024C023C022C021D020E020001F206
:10615D0001E401D701CA01BE01B101A6019A018F67
:10616D000185017A01700166015D0153014A01410A
:10617D00013901310129012101190112010B01041C
:10618D0000FD00F700F000EA00E400DE00D900D3C6
:10619D0000CE00C900C400BF00BA00B500B100AD0B
:1061AD0000A800A400A0009C009900950091008E0D
:0C61BD00008A008700840081007E007BC7
:10009E007547009007BAE4F0A3F075310075300093
:1000AE00754D00754E00C235D23674FE9007BCF801
:1000BE00E4F0E8A3F074FE9007BEF8E4F0E8A3F0D5
:1000CE0074FE9007C8F0745A9007C9F0745A9007DE
:1000DE00CAF0D237C229C239C23422750B00750A52
:1000EE0000AE0AAF0BAC08AD09EDC39FEC9E4016F7
:1000FE0074FF12657575CF01780B740126F65004E6
:10010E0018E436F650DB22900041E0B4AA1C9007AA
:10011E0076E0B43C159007B6E0FEA3E0FFEF4E602C
:10012E0009741EBE0004D39F5003020243755D0086
:10013E00755C0075F8099007B6E0FEA3E0FF740742
:10014E006F4E6006740E6F4E7006743A900776F01E
:10015E009007B6E0FEA3E0FF7408BE001ED39F40DA
:10016E001A7E017F089007B6E0FCA3E0FD1DBDFFDF
:10017E00011C1200038E5A8F5B801F9007B6E0FEA3
:10018E00A3E0FF74081265D98F048E057E017F08E7
:10019E00CDCCCD1200038E5A8F5BAE5CAF5D740C6E
:1001AE00D39F74019E500302023EA2F9B3407EE536
:1001BE005D455C700375A382AE5CAF5D74016F4EDE
:1001CE00700375A300AE5CAF5D74026F4E700D9040
:1001DE0007B7E075F002A4FDACF08DA3AE5CAF5D89
:1001EE0074036F4E700375A300AE5CAF5D7403BEF7
:1001FE0000039F5013AC5AAD5BED2FFFEC3EFE900B
:10020E0000721265BCE0F5A3AE5CAF5DEFB40B09F6
:10021E00EEB401057414126575AE5CAF5DEFB40BF0
:10022E0007EEB4010375F80D785C1265E90201A8BA
:10023E00900041E4F022755D00755C0075F8099040
:10024E0007B6E0FEA3E0FF7408BE001ED39F401A5F
:10025E007E017F089007B6E0FCA3E0FD1DBDFF0107
:10026E001C1200038E5A8F5B801F9007B6E0FEA310
:10027E00E0FF74081265D98F048E057E017F08CDCC
:10028E00CCCD1200038E5A8F5BAE5CAF5D7411D372
:10029E009F74019E5003020374A2F9B3500302032C
:1002AE0071E55D455C700375A3D2AE5CAF5D740104
:1002BE006F4E700375A300AE5CAF5D74026F4E702F
:1002CE000D9007B7E075F002A4FDACF08DA3AE5C07
:1002DE00AF5D74036F4E700375A300AE5CAF5D74BB
:1002EE00046F4E700375A300AE5CAF5D74056F4E68
:1002FE00700375A300AE5CAF5D74066F4E70037530
:10030E00A300AE5CAF5D74076F4E700375A300AEB5
:10031E005CAF5D74086F4E700375A300AE5CAF5D8D
:10032E007408BE00039F5016AC5AAD5BED2FFFEC68
:10033E003EFE90006D1265BCE5A3F075A300AE5CA9
:10034E00AF5DEFB41009EEB401057414126575AE0D
:10035E005CAF5DEFB41007EEB4010375F80D785C79
:10036E001265E902029722755D00755C0075F80949
:10037E00AE5CAF5D7417BE0004D39F500302044DF4
:10038E00A2F9B3500302044AE55D455C700375A300
:10039E00D2AE5CAF5D74016F4E700375A300AE5CA0
:1003AE00AF5D74026F4E700D9007B7E075F002A44A
:1003BE00FDACF08DA3AE5CAF5D74036F4E70037534
:1003CE00A300AE5CAF5D74046F4E700375A300AEF8
:1003DE005CAF5D74056F4E700375A300AE5CAF5DD0
:1003EE0074066F4E700375A300AE5CAF5D74076F3D
:1003FE004E700375A300AE5CAF5D74086F4E700354
:10040E0075A300AE5CAF5D7408BE00039F500C90E8
:10041E00004F1265BCE5A3F075A300AE5CAF5D7432
:10042E00166F4E70057414126575AE5CAF5D741662
:10043E006F4E700375F80D785C1265E902037E222B
:10044E00900041E0B4AB0280030204E8755D0075D4
:10045E005C0075F809AE5CAF5D7412BE007CD39F74
:10046E004078A2F9B34070E55D455C700375A382D8
:10047E00AE5CAF5D74016F4E700375A300AE5CAFE2
:10048E005D74026F4E700D9007B7E075F002A4FD1B
:10049E00ACF08DA3AE5CAF5D74036F4E700375A3AD
:1004AE0000AE5CAF5D7403BE00039F500990005414
:1004BE001265BCE0F5A3AE5CAF5D74116F4E7005B6
:1004CE007414126575AE5CAF5D74116F4E7003756A
:1004DE00F80D785C1265E9020463229007C5E4F01A
:1004EE0074649007B6F8E4F0E8A3F012037574C8CC
:1004FE009007B6F8E4F0E8A3F074FF90004FF074A4
:10050E00FF900050F074FF900051F074009000497D
:10051E00F074FF900052F07400900054F07401904B
:10052E000055F090005BE0B4371A900058E0900050
:10053E004FF0900059E0900050F090005AE090007B
:10054E0051F080469007C57401F074659007B6F8B7
:10055E00E4F0E8A3F012037574C89007B6F8E4F05F
:10056E00E8A3F090005BE0B4371A900058E09000DA
:10057E004FF0900059E0900050F090005AE090003B
:10058E0051F0800674029007C5F09007C6E4F0742F
:10059E00669007B6F8E4F0E8A3F012037574C890FD
:1005AE0007B6F8E4F0E8A3F090005AE0B4371290E2
:1005BE000058E0900049F0900059E0900052F08011
:1005CE00769007C67401F074679007B6F8E4F0E809
:1005DE00A3F012037574C89007B6F8E4F0E8A3F020
:1005EE0090005AE0B43712900058E0900049F09015
:1005FE000059E0900052F0803E74029007C6F074ED
:10060E00689007B6F8E4F0E8A3F012037574C8908A
:10061E0007B6F8E4F0E8A3F090005AE0B437129071
:10062E000058E0900049F0900059E0900052F080A0
:10063E000674039007C6F022E54E64046006E59941
:10064E0064FF60028031A2354004D2358027E54E2A
:10065E00600874E6254E900045F0E54D600874F094
:10066E00254D900045F0E54EB4010280FE754E001A
:10067E00754D00C2358002C235E54E90384AF828D5
:10068E002873754E00E599B4FF03754D01E599B4D5
:10069E00FE03754D02E599B4FD03754D03E599B45E
:1006AE00FC03754D04E599B4FA03754D05E599B44F
:1006BE00FB06754E01124015E599B4F906754E0408
:1006CE00124015E599D394E54007E599C394F0409F
:1006DE0002801685994F754E027E017F00E54FC34D
:1006EE0094E61265958E328F339007BAE4F0A3F03C
:1006FE00E599D394C44007E599C394E64002802857
:10070E0085994F754E0374E5C3954FF533753200D9
:10071E00AE32AF33905E6D126564E493F87401935C
:10072E009007BAC8F0A3C8F0D299020C56900058A0
:10073E00E07005A227B3400280429007BAE0FEA304
:10074E00E0FF74FFBE00039F5009EFC39446EE9482
:10075E000640119007BAE0FEA3E0FFEFD3946DEED2
:10076E00940640139007BAE0FEA3E0FF90007612C5
:10077E0065BCE599F0800385997480119007BAE005
:10078E00FEA3E0FF9000761265BCE599F09007BAE3
:10079E001265A39007BAE0FEA3E0FFEFB40106EEE8
:1007AE00B4070280030209FD900776E0B43C028094
:1007BE00030209FDA22750030208E8C29C900058CC
:1007CE00E0900114F0900059E0900083F090005AF0
:1007DE00E09000A3F090005BE09000CCF090005C05
:1007EE00E0900078F090005DE09000BEF090005E2A
:1007FE00E09000DCF090005FE09000B0F0900060C0
:10080E00E09000CEF0900061E09000FEF09000626B
:10081E00E0900162F0900063E0900163F09000645C
:10082E00E0900164F0123B8690006AE09000E5F0E3
:10083E0090006BE090009CF090006CE090009DF0BA
:10084E0074639007B6F8E4F0E8A3F074AB9000413F
:10085E00F012044E900041E4F07464F5097508003E
:10086E001200E9A21C4039757301E573D394075049
:10087E002DE5739007B6F8E4F0E8A3F074AA9000A3
:10088E0041F0120115E573C39407500A7464F5091B
:10089E007508001200E97873740126F650CC803783
:1008AE00757308E573D3940E502DE5739007B6F863
:1008BE00E4F0E8A3F074AA900041F0120115E5737C
:1008CE00C3940E500A7464F5097508001200E97895
:1008DE0073740126F650CC0209E7C29C900114E015
:1008EE00900058F0900083E0900059F09000A3E043
:1008FE0090005AF09000CCE090005BF0900078E011
:10090E0090005CF09000BEE090005DF09000DCE0A6
:10091E0090005EF09000B0E090005FF09000CEE0AE
:10092E00900060F09000FEE0900061F07400900086
:10093E0062F07400900063F07400900064F07463D1
:10094E009007B6F8E4F0E8A3F074AB900041F01213
:10095E00044E900041E4F07464F50975080012002D
:10096E00E9757301E573D394075026E5739007B6C6
:10097E00F8E4F0E8A3F074AA900041F012011574A7
:10098E0064F5097508001200E97873740126F650B3
:10099E00D3D29C7599FB743C900776F0757308E57D
:1009AE0073D3940E5026E5739007B6F8E4F0E8A3DF
:1009BE00F074AA900041F01201157464F5097508DF
:1009CE00001200E97873740126F650D374C89007AC
:1009DE00B6F8E4F0E8A3F080FE74C89007B6F8E429
:1009EE00F0E8A3F0D29C754E00754D007599FB0290
:1009FE000C569007BAE0FEA3E0FFEF4E7006859905
:100A0E00317530009007BAE0FEA3E0FF74016F4E1F
:100A1E00701BAC30AD31AA32AB33ED2BFBEC3AFA96
:100A2E008A068B079000761265BCE599F09007BA9E
:100A3E001265A39007BAE0FEA3E0FF74026F4E703A
:100A4E0021AC30AD3174566D4C7006E54F64E660E6
:100A5E00028003124015123B86854F99754E007524
:100A6E004D00020C569007BAE0FEA3E0FF90007610
:100A7E001265BCE599F09007BA1265A39007BAE02B
:100A8E00FEA3E0FFAC32AD338F028E038C068D07D2
:100A9E00905EB1126564E493F9740193FEEAD39EFD
:100AAE00EB994009854F99754E00754D00020C5615
:100ABE009007BAE0FEA3E0FF9000761265BCE599C0
:100ACE00F09007BA1265A39007BAE0FEA3E0FFEF1D
:100ADE00B40006EEB401028003020C56900051E001
:100AEE00D394C7400B900051E0C394C8F550801AC0
:100AFE00900051E0D39463400B900051E0C3946496
:100B0E00F5508006900051E0F550E55075F002A4C6
:100B1E00FFAEF08F73EF9000761265C7EFFCE0FD2D
:100B2E00EC9000791265C7EDFCE0FDEC2DB550029E
:100B3E008003020C470FEF9000761265C7E573FF36
:100B4E00E0FCEF90007A1265C7ECFFE0FCEFC39C6F
:100B5E00B550028003020C47E5739000781265C70A
:100B6E00E573FFE0FCEF90007B1265C7ECFFE0FC45
:100B7E00EF2CB550028003020C47E57390007C12F7
:100B8E0065C7E0C39550900058F0E57390007D1254
:100B9E0065C7E0C39550900059F0E57390007E1242
:100BAE0065C7E0C3955090005AF0740090005BF05A
:100BBE0074FF90005CF0E5739000801265C7E0C38F
:100BCE00955090005DF0E5739000811265C7E0C30B
:100BDE00955090005EF0E5739000821265C7E0C3F9
:100BEE00955090005FF0E57390007F1265C7E0C3EB
:100BFE0095509007B6F8E4F0E8A3F074AB9000417E
:100C0E00F012044E7464F5097508001200E990079D
:100C1E00B61265A312044E7464F50975080012002D
:100C2E00E99007B61265A312044E7599F97464F52E
:100C3E00097508001200E980FE7599FF7464F509C4
:080C4E007508001200E980FEA8
:0F384A0002069002073B020A00020A73020ABE3E
:100C560022E54D903859F8282873020D699007BA95
:100C6600E0FEA3E0FF9000471265BCE0F59990070F
:100C7600BA1265A39007BAE0FEA3E0FF74116F4EA7
:100C86007003754D00020D69856E99020D69900716
:100C9600BAE0FEA3E0FF9000761265BCE0F599EF9E
:100CA600B40107EEB40703754D009007BA1265A3A9
:070CB600020D699007BBE08D
:0F385900020C60020C63020C8E020C94020CB97C
:100CBD00903A0CF8282873855399020D5E855F993B
:100CCD00020D5E856199020D5E856599020D5E8549
:100CDD006799807D85689980788569998073856A23
:100CED0099806E900016E0F5998066A236B34007A4
:100CFD007599FAC2368041A226B3400575990F80C9
:100D0D00359007C5E0600A9007C5E024DCF59980B1
:100D1D00169007C6E0600A9007C6E024DEF59980BC
:100D2D0006900045E0F599900045E4F09007C5E484
:100D3D00F09007C6E4F0C2268017856B9980128566
:100D4D006699800D856C9980087599FC8003754DA9
:010D5D000095
:103A0C00020CC4020CCA020CD0020CD6020CDC0252
:103A1C000CE1020CE6020CEB020CF0020CF8020DAD
:0D3A2C0047020D4C020D51020D56020D5BBC
:0B0D5E009007BA1265A38003123A3917
:03386800020D66E8
:100D690022E537255BFFAE5A50010E9000761265D9
:100D7900BCE0F538E537255BFFAE5A50010E0FBFD1
:100D890000010E9000761265BCE0F539853F3BE520
:100D990038B539058538378041E539D39538401D4F
:100DA900E539C39538853AF0A4FFAEF0E53B8E04EA
:100DB9008F05FF126585ED2538F537801DE538C3A8
:100DC9009539853AF0A4FFAEF0E53B8E048F05FF17
:100DD900126585EDF4042538F53722E539D39538C0
:100DE900401DE539C39538853AF0A4FFAEF0E53BDF
:100DF9008E048F05FF126585ED2538F537801DE5D1
:100E090038C39539853AF0A4FFAEF0E53B8E048FDF
:100E190005FF126585EDF4042538F5372290007C2D
:100E2900E0B40170E56775F00A84FF7E008F37E54D
:100E39006775F00A84ADF07C008D3A753F0A755AE2
:100E490005755B24E537C394115005120D6A8006B8
:100E59009005ABE0F537E53790006FF0E56775F081
:100E69000A84FF7E008F37E56775F00A84ADF07C50
:100E7900008D3A753F0A755A05755B5AE537C39473
:100E8900115005120D6A80069005E1E0F537E53746
:100E990090000EF02290007CE0B4016AE56775F0DD
:100EA9000A84FF7E008F37E56775F00A84ADF07C10
:100EB900008D3A753F0A755A05755B36E537C39457
:100EC900115005120D6A80069005BDE0F53785378A
:100ED9004BE56775F00A84FF7E008F37E56775F08B
:100EE9000A84ADF07C008D3A753F0A755A05755B29
:100EF90048E537C394115005120D6A80069005CF55
:100F0900E0F53785374C22E55F75F00484FF7E00F4
:100F19008F37E55F75F00484ADF07C008D3A753F3D
:100F290004755A01755B00E537C3943F5005120DEE
:100F39006A80069001B5E0F5378537297528009054
:100F49000044E075F020A4FFAEF09000C7E08E04E5
:100F59008F05FF1265858D379000AFE0D3955F50FF
:100F6900030210169000D3E0D3955F4010ED900175
:100F7900B61265C7E0F52B752A0002101390009E82
:100F8900E0D3955F4043E5379001B61265C7E0F5B8
:100F990038E5379001D61265C7E0F5399000D3E0FE
:100FA900F404255FF53A90009EE0FE9000D3E0F44A
:100FB900042EF53BE538B539058538378003120D20
:100FC900E485372B752A008041E5379001D61265F3
:100FD900C7E0F538E5379001F61265C7E0F53990B5
:100FE900009EE0F404255FF53A9000AFE0FE900022
:100FF9009EE0F4042EF53BE538B539058538378090
:1010090003120DE485372B752A000210BD9000D616
:10101900E0D3955F5011E5379002361265C7E0F5C8
:101029002B752A000210BD90009FE0D3955F5043B5
:10103900E5379002161265C7E0F538E537900236B4
:101049001265C7E0F53990009FE0F404255FF53A91
:101059009000D6E0FE90009FE0F4042EF53BE538C1
:10106900B539058538378003120DE485372B752A84
:10107900008041E5379001F61265C7E0F538E5379C
:101089009002161265C7E0F5399000AFE0F4042527
:101099005FF53A90009FE0FE9000AFE0F4042EF572
:1010A9003BE538B539058538378003120DE48537B6
:1010B9002B752A00229000E7E0F53C753F11755A1F
:1010C90002755B00AE52AF53E53C75F00FA4FDAC61
:1010D900F0EDD39FEC9E4021E53C8E048F05FF1275
:1010E9006585ED75F010A4FFAEF0E55F75F011842C
:1010F900FD7C00ED2FF53D800EE55F75F01184FF55
:101109007E00EF24F0F53D853D37E55F75F01184EC
:10111900AFF07E008F3A120D6A85373EAE52AF535B
:101129009000E7E075F00FA4FDACF0EDD39FEC9EC5
:101139004028755A02755B10853D37120D6A853E48
:1011490038853739AE52AF53E53C8E048F05FF120F
:1011590065B08D3A853C3B120DE485372975280029
:10116900752B64752A00229000E7E0F53C753F1164
:10117900755A02755B00AE52AF53E53C75F00FA48A
:10118900FDACF0EDD39FEC9E4021E53C8E048F052C
:10119900FF126585ED75F010A4FFAEF0E56175F0FD
:1011A9001184FD7C00ED2FF53D800EE56175F01190
:1011B90084FF7E00EF24F0F53D853D37E56175F04C
:1011C9001184AFF07E008F3A120D6A85373EAE5218
:1011D900AF539000E7E075F00FA4FDACF0EDD39F9D
:1011E900EC9E4028755A02755B10853D37120D6AD1
:1011F900853E38853739AE52AF53E53C8E048F05AD
:10120900FF1265B08D3A853C3B120DE4853729758F
:101219002800E56B6017E56BC394FE50109000DB66
:10122900E0B402099000C9E0D3940B50028017AED4
:1012390028AF29E56B12659574E78E048F05FF12B7
:1012490065858C288D299000B1E0B40453E55F755C
:10125900F00484FF7E008F37E55F75F00484ADF0FC
:101269007C008D3A753F04755A01755B00E537C3FB
:10127900943F5005120D6A80069001B5E0F537AE2E
:1012890028AF29E53712659574648E048F05FF121E
:101299006585AE28AF29EF2DFDEE3CFC8C288D2904
:1012A900752B64752A002290007CE0B40146E5673D
:1012B90075F00A84FF7E008F37E56775F00A84AD03
:1012C900F07C008D3A753F0A755A05755B00E53764
:1012D900C394115005120D6A8006900587E0F53711
:1012E900AE2AAF2BE5372FFF50010E74641265D972
:1012F9008E2A8F2B90007DE0B40146E56875F00ACF
:1013090084FF7E008F37E56875F00A84ADF07C00B4
:101319008D3A753F0A755A05755B6CE537C39411AB
:101329005005120D6A80069005F3E0F537AE2AAF35
:101339002BE5372FFF50010E74641265D98E2A8F61
:101349002B90008CE0B40249E56AC3944175F0051D
:1013590084FF7E008F37E56A75F00584ADF07C0067
:101369008D3A753F05755A06755B00E537C39413C9
:101379005005120D6A8006900689E0F537AE2AAF4E
:101389002BE5372FFF50010E74641265D98E2A8F11
:101399002B9000CEE0B40202800302144FE55F7582
:1013A900F01584FF7E008F37E55F75F01584ADF089
:1013B9007C008D3A753F15755A03755BF4E537C3A3
:1013C900940B5005120D6A8006900475E0F537E517
:1013D9003775F0FFA4FFAEF09000CFE08E048F05C3
:1013E900FF126585ED900068F0E56675F078A4FF59
:1013F900AEF074FF8E048F05FF1265858C5A8D5BE4
:1014090074028C068D071200398F37AC5AAD5B74A4
:1014190004FF1265B08D3A753F04755A06755B284D
:10142900E537C3941D5005120D6A80069006BBE08E
:10143900F537AE2AAF2BE5372FFF50010E74641232
:1014490065D98E2A8F2B90007BE0B4025DE561752A
:10145900F064A4FFAEF074081200398E5C8F5D74DD
:10146900058E048F05FF1265858D37AE5CAF5D74FF
:10147900058E048F05FF1265B08D3A753F05755AC3
:1014890005755BDEE537C394135005120D6A8006B6
:10149900900667E0F537AE2AAF2BE5372FFF5001ED
:1014A9000E74641265D98E2A8F2B9000BDE0703CB2
:1014B900900044E075F00584FF7E008F379000446A
:1014C900E075F00584ADF07C008D3A753F05755ADD
:1014D90005755BC0E537C3941D5005120D6A80067A
:1014E900900653E0F537E537900070F022900084BC
:1014F900E0B401179007C1E0252BFFAE2A50010E79
:101509009000D8E01265D98E2A8F2B9000FCE0B4A8
:1015190001149000FDE0A852B8000495535007E566
:101529005FC39560400280129000A6E0252BFFAEB4
:101539002A50010E8E2A8F2B802F900084E0B4034D
:1015490016A229B3B350109007C4E0C39405A8525A
:10155900B800069553400280109000A6E0252BFFA5
:10156900AE2A50010E8E2A8F2B90007EE0B4020223
:1015790080030218F4900081E0602FE567D3944658
:10158900402890000FE0FEA3E0FF9000BCE075F05A
:1015990003A4FDACF0EFD39DEE9C400E9000E0E07B
:1015A900A852B80005D3955350030218F49000B11E
:1015B900E0B40302800302175885615B755A0090F5
:1015C9000088E0A852B800049553500E900089E0B5
:1015D900A85AB80005D3955B5003021755E5617504
:1015E900F002A4FFAEF074158E048F05FF12658515
:1015F9008C068D079006061265BCFEE0FFEE900092
:1016090080E0FEEF8E0088F0A4FFAEF074648E04D3
:101619008F05FF1265858C5A8D5B900044E075F04B
:1016290018A4FFAEF09000C7E08E048F05FF126585
:10163900858C068D0790061E1265BCAE5AAF5BE01D
:1016490012659574648E048F05FF1265858C5A8D19
:101659005BE565A85AB80077D3955B4072E565C329
:10166900955BFFE4955AFE8E5A8F5B7428BE000382
:101679009F500C755B28755A00740D900045F0AEAB
:101689005AAF5B900081E012659574288E048F052E
:10169900FF1265858C5A8D5BAE28AF29740A8E04BA
:1016A9008F05FF1265858D068C07AC5AAD5BCFCED1
:1016B900CF120003740A8E048F05FF1265858C5AB8
:1016C9008D5BAE28AF291265E18E288F29807DE5D3
:1016D90065A85AB80004955B5072AE5AAF5BE565D0
:1016E9001265D98E5A8F5B7428BE00039F500C7502
:1016F9005B28755A00740D900045F0AE5AAF5B90A7
:101709000081E012659574288E048F05FF126585A6
:101719008C5A8D5BAE28AF29740A8E048F05FF128F
:1017290065858D068C07AC5AAD5BCFCECF12000311
:10173900740A8E048F05FF1265858C5A8D5BAE285D
:10174900AF29EF2DFDEE3CFC8C288D290218F49071
:1017590000C9E0855FF0A4FFAEF0740512659574C9
:10176900071200398E5A8F5B900088E0A852B800A2
:101779000495535012900089E075F002A4FDACF075
:10178900EFC39DEE9C40030218F4E55F75F00B84EE
:10179900FF7E009006061265BCFEE0FFEE90008019
:1017A900E0FEEF8E0088F0A4FFAEF074648E048F23
:1017B90005FF1265858C5A8D5B900044E075F01821
:1017C900A4FFAEF09000C7E08E048F05FF12658577
:1017D9008C068D0790061E1265BCAE5AAF5BE012EF
:1017E900659574648E048F05FF1265858C5A8D5B2F
:1017F900E565A85AB80077D3955B4072E565C3954E
:101809005BFFE4955AFE8E5A8F5B7428BE00039FD6
:10181900500C755B28755A00740D900045F0AE5A4E
:10182900AF5B900081E012659574288E048F05FFE7
:101839001265858C5A8D5BAE28AF29740A8E048F88
:1018490005FF1265858D068C07AC5AAD5BCFCECFEF
:10185900120003740A8E048F05FF1265858C5A8D58
:101869005BAE28AF291265E18E288F29807DE56559
:10187900A85AB80004955B5072AE5AAF5BE5651281
:1018890065D98E5A8F5B7428BE00039F500C755B17
:1018990028755A00740D900045F0AE5AAF5B900060
:1018A90081E012659574288E048F05FF1265858C79
:1018B9005A8D5BAE28AF29740A8E048F05FF126515
:1018C900858D068C07AC5AAD5BCFCECF1200037461
:1018D9000A8E048F05FF1265858C5A8D5BAE28AF81
:1018E90029EF2DFDEE3CFC8C288D29229000DCE0AF
:1018F900B4026AE55F75F00884FF7E008F37E55F03
:1019090075F00884ADF07C008D3A753F08755A0171
:10191900755BE0E537C3943F5005120D6A80069068
:101929000275E0F53785372D752C00AE2CAF2DAC3F
:101939002AAD2B12000374648E048F05FF1265858E
:101949008C2C8D2D900079E08C068D07126595748D
:10195900648E048F05FF1265858C2C8D2DAE28AF02
:1019690029AC2AAD2B12000374648E048F05FF1273
:1019790065858C288D29900079E08C068D07126584
:101989009574648E048F05FF1265858C288D29A2B4
:101999000D401DAE52AF537405BE00039F5002D2D5
:1019A9000DE561D394CC4008D2017411900045F043
:1019B9009000DBE0B402089000C9E0640B6002808B
:1019C90035AE28AF29E56B12659574E78E048F054E
:1019D900FF1265858C288D299000DCE0B40217AED2
:1019E9002CAF2DE56B12659574E78E048F05FF12F8
:1019F90065858C2C8D2D90009BE05402601B900016
:101A090092E0A852B80012D39553400DA20DB3B37A
:101A19005007E561C3949A40028028AE34AF3590EF
:101A29000090E075F002A4FDACF0EF2DFDEE3CFC5A
:101A390074022DFD50010CE561BC0007D39D4003E4
:101A4900754301856135753400E5437003021B3820
:101A59009000EEE0C395435003021B2A9000FEE07C
:101A6900C394025076E56775F00A84FF7E009005FD
:101A7900761265BCE0F55B755A00AE5AAF5B900013
:101A890091E012659574648E048F05FF1265858C4B
:101A99005C8D5D9000EEE004C395438C068D0712C2
:101AA90065959000EEE08E048F05FF1265858C5CCC
:101AB9008D5DAE28AF29EF2DFDEE3CFC8C288D29DC
:101AC9009000DCE0B40212AE2CAF2DAA5CAB5DEF46
:101AD9002BFBEE3AFA8A2C8B2D80469000EEE0041F
:101AE900C39543854BF0A4FFAEF09000EEE08E0461
:101AF9008F05FF1265858C5C8D5DAE28AF29EF2DB2
:101B0900FDEE3CFC8C288D299000DCE0B40212AE7D
:101B19002CAF2DAA5CAB5DEF2BFBEE3AFA8A2C8B2E
:101B29002D05439000EEE0C39543500375430090A3
:101B3900009BE05401601B90008FE0A852B800128E
:101B4900D39553400DA20DB3B35007E55FC394CCB1
:101B59004002802590008DE075F003A4FFAEF0E50A
:101B6900402FFF50010E74032FFF50010EE55FBE99
:101B79000007D39F4003754401855F40E544700326
:101B8900021C6B9000EFE0C395445003021C5D906A
:101B990000FEE0C394025076E56775F00A84FF7E83
:101BA900009005761265BCE0F55B755A00AE5AAF38
:101BB9005B90008EE012659574648E048F05FF12A8
:101BC90065858C5C8D5D9000EFE004C395448C06BF
:101BD9008D071265959000EFE08E048F05FF126561
:101BE900858C5C8D5DAE28AF29EF2DFDEE3CFC8C1C
:101BF900288D299000DCE0B40212AE2CAF2DAA5C2E
:101C0900AB5DEF2BFBEE3AFA8A2C8B2D80469000C8
:101C1900EFE004C39544854CF0A4FFAEF09000EFCB
:101C2900E08E048F05FF1265858C5C8D5DAE28AF53
:101C390029EF2DFDEE3CFC8C288D299000DCE0B4C9
:101C49000212AE2CAF2DAA5CAB5DEF2BFBEE3AFA7C
:101C59008A2C8B2D05449000EFE0C3954450037501
:101C690044009000F1E02529FFAE2850010E8E288E
:101C79008F299000A0E0A828B80004952950099060
:101C890000A0E0F5297528009000DCE0B4020D9071
:101C990000A0E0A82CB80006952D4002800990000C
:101CA900A0E0F52D752C00229000DCE0B401028043
:101CB90003021DBCA20DB35003021DBA9000A7E098
:101CC900B40168AE28AF29AC52AD53120003743C7D
:101CD9008E048F05FF1265859000B7E0BC00109D4A
:101CE900400D9000B9E0A828B8000495295002D207
:101CF90002AE28AF29AC52AD53120003743C8E04D6
:101D09008F05FF1265859000B7E0C3940ABC0015E2
:101D1900D39D40119000B9E0C39405A828B80005E7
:101D2900D3952950028002C2028068AE28AF29AC3F
:101D390052AD5312000374788E048F05FF12658526
:101D49009000B7E0BC00109D400D9000B9E0A828B4
:101D5900B8000495295004D2028038AE28AF29ACC6
:101D690052AD5312000374788E048F05FF126585F6
:101D79009000B7E0C3940ABC0015D39D40119000B0
:101D8900B9E0C39405A828B80005D3952950028065
:101D990002C202A202B34019AE28AF299000B8E0EE
:101DA90012659574648E048F05FF1265858C288DE4
:101DB900298002C202A200B34006A201B3B35009AE
:101DC900900015E4F0A3F08024AE28AF297400D365
:101DD9009F74019E400C900015E528F0A3E529F0B9
:101DE900800B74FF900015F8E4F0E8A3F09000BEB2
:101DF900E0D39402400C9000A9E07006A20DB3B3A1
:101E09004002801AAE28AF2974021265958E288F78
:101E190029AE2CAF2D74021265958E2C8F2D900052
:101E2900A7E0B4011AAE28AF2974021265958E286D
:101E39008F29AE2CAF2D74021265958E2C8F2DAE85
:101E490028AF29745E126595740A8E048F05FF12F6
:101E590065858C288D299000DCE0B40217AE2CAF83
:101E69002D745E126595740A8E048F05FF126585BF
:101E79008C2C8D2DAE28AF297402BE000AD39F4049
:101E890006752902752800AE2CAF2D7402BE000A12
:101E9900D39F4006752D02752C00900013E528F09C
:101EA900A3E529F022900044E09003761265C7E08B
:101EB900F541754264900044E0FE9000B2E0D39E83
:101EC9004037E55F75F00884FF7E008F37E55F7561
:101ED900F00884ADF07C008D3A753F08755A03759A
:101EE9005B96E537C3941F5005120D6A800690046E
:101EF9002BE0F5378537428035E55F75F00884FFBB
:101F09007E008F37E55F75F00884ADF07C008D3A6F
:101F1900753F08755A03755BB6E537C3941F5005BD
:101F2900120D6A800690044BE0F5378537422290FE
:101F390000E8E0F53C753F11755A04755B00AE5237
:101F4900AF53E53C75F00FA4FDACF0EDD39FEC9ECB
:101F59004021E53C8E048F05FF126585ED75F01073
:101F6900A4FFAEF0E55F75F01184FD7C00ED2FF55F
:101F79003D800EE55F75F01184FF7E00EF24F0F5DA
:101F89003D853D37E55F75F01184AFF07E008F3AEE
:101F9900120D6A85373EAE52AF539000E8E075F0F6
:101FA9000FA4FDACF0EDD39FEC9E4028755A047543
:101FB9005B10853D37120D6A853E38853739AE523B
:101FC900AF53E53C8E048F05FF1265B08D3A853C11
:101FD9003B120DE4853741754264229000E8E0F533
:101FE9003C753F11755A04755B00AE52AF53E53C21
:101FF90075F00FA4FDACF0EDD39FEC9E4021E53CBC
:102009008E048F05FF126585ED75F010A4FFAEF003
:10201900E56175F01184FD7C00ED2FF53D800EE53D
:102029006175F01184FF7E00EF24F0F53D853D37A1
:10203900E56175F01184AFF07E008F3A120D6A8563
:10204900373EAE52AF539000E8E075F00FA4FDACF7
:10205900F0EDD39FEC9E4028755A04755B10853DC1
:1020690037120D6A853E38853739AE52AF53E53C94
:102079008E048F05FF1265B08D3A853C3B120DE445
:102089008537417542649000B1E0B4047990004409
:10209900E0FE9000B2E0D39E4037E55F75F008841A
:1020A900FF7E008F37E55F75F00884ADF07C008D09
:1020B9003A753F08755A03755B96E537C3941F5007
:1020C90005120D6A800690042BE0F53785374280AA
:1020D90035E55F75F00884FF7E008F37E55F75F0A1
:1020E9000884ADF07C008D3A753F08755A03755B1D
:1020F900B6E537C3941F5005120D6A800690044B4C
:10210900E0F5378537422290007CE0B4013BE56772
:1021190075F00A84FF7E008F37E56775F00A84AD94
:10212900F07C008D3A753F0A755A05755B12E537E3
:10213900C394115005120D6A8006900599E0F53790
:10214900E5422537C39464F54290007DE0B4013B34
:10215900E56875F00A84FF7E008F37E56875F00A37
:1021690084ADF07C008D3A753F0A755A05755B7E22
:10217900E537C394115005120D6A8006900605E0F3
:10218900F537E5422537C39464F542E5412542F523
:1021990036900084E0B402109007C0E02536FE9026
:1021A90000D8E0F4042EF5369000DBE0D39401402A
:1021B90040E56BC394E7501D74E7C3956BFE900728
:1021C900C2E08E00F5F0E884FF7E008F37E5362502
:1021D90037F536801CE56BC394E7FE9007C2E08EA5
:1021E90000F5F0E884FF7E008F37E536C39537F5B3
:1021F90036A20D4006E5412464F536E536D39464EC
:102209004009E536C39464F53680037536009000BD
:10221900B4E0C3953650069000B4E0F53622D200FA
:1022290090006EE0A852B800049553504190006E9A
:10223900E0A852B800049553500375360F90006E0C
:10224900E004A852B800049553500375360A90006B
:102259006EE02402A852B80004955350057536055E
:10226900C20090006EE060067409900045F0C23922
:102279007E017F009000BAE01265959000C9E08E5A
:10228900048F05FF126585E55FBC0017D39D4013D8
:102299009000C3E0B40204D2398002C200740A90EB
:1022A9000045F09000BBE0C3956750159000CDE064
:1022B900A852B8000495535002C200740B9000450F
:1022C900F0E567C39464501D900113E0600D90011F
:1022D90013E0A852B80006955340028008C2007462
:1022E9000B900045F0A20040037536059000FCE014
:1022F900B401149000FDE0A852B8000495535007AA
:10230900E55FC39560400280089000A5E0F536803E
:102319003A900084E0B40306A229B3B34002802BAB
:102329009007C4E0C39405A852B800049553500C13
:102339009000A5E0F536740C900045F09007C4E0D4
:10234900A852B8000495535002C20085366C90001B
:1023590076E02536FE900044E075F01E84FC7F008F
:10236900EE2CF53622900044E075F00584FF7E00DE
:102379008F37900044E075F00584ADF07C008D3A0C
:10238900753F05755A03755BD69000C7E01475F063
:102399000584FF7E00E537BE00039F5005120D6AD4
:1023A900800BE53790044C1265C7E0F537E53790A7
:1023B90007C3F09007C3E0FE9000B6E0C39E500843
:1023C9009000B6E09007C3F022E56775F00A84FF34
:1023D9007E009005761265BCE0F546E546D3946427
:1023E9004010E546C3946475F00F84FF7E008F4664
:1023F9008003754600900099E02546F54622900035
:10240900B1E0C3940350269007B0E0FEA3E0FF7447
:1024190004120039E55F126595740F8E048F05FF6C
:102429001265859007AEECF0A3EDF080249007B01B
:10243900E0FEA3E0FF7404120039E56112659574AA
:102449000F8E048F05FF1265859007AEECF0A3EDA2
:10245900F090008CE0B40262E56AC3944175F0051E
:1024690084FF7E008F37E56A75F00584ADF07C0046
:102479008D3A753F05755A06755B14E537C3941790
:102489005005120D6A800690069DE0F5379007AE5B
:10249900E0FEA3E0FF740A8E048F05FF126585E54F
:1024A900378C068D07126595740A8E048F05FF1205
:1024B90065859007AEECF0A3EDF09007AEE0FEA3C2
:1024C900E0FF9007B4E0FCA3E0FDEDD39FEC9E4054
:1024D9000F9007B4E0F8A3E09007AEC8F0A3C8F0E6
:1024E900229006BDE090386BF8282873804C8553FC
:1024F9007380479000C9E0855FF0A4FFAEF07408CF
:102509001200398F738033856173802E85677380DC
:10251900298568738024856973801F856A73801A89
:10252900856B7380158566738010856573800B854F
:0A2539006C738006900016E0F57345
:10386B000224F50224F70224FC022510022515027E
:10387B00251A02251F02252402252902252E0225A1
:07388B003302253802253D40
:102543009006BEE0FE9006BFE0D39E404B9006BDD2
:10255300E0B404189006BFE0C395735002D22A90EA
:1025630006BEE0D395734002C22A802A9006BEE0DD
:10257300C3957350099006BFE0D395735002800250
:10258300D22A9006BEE0D3957350099006BFE0C3EC
:1025930095735002C22A802A9006BEE0D3957340F9
:1025A300099006BFE0C3957340028002C22A9006D9
:1025B300BEE0C3957340099006BFE0D39573400214
:1025C300D22A229006C1E0903892F8282873804CD2
:1025D30085537380479000C9E0855FF0A4FFAEF098
:1025E30074081200398F738033856173802E856779
:1025F3007380298568738024856973801F856A7356
:10260300801A856B7380158566738010856573806A
:0C2613000B856C738006900016E0F573D8
:103892000225D10225D30225D80225EC0225F10208
:1038A20025F60225FB02260002260502260A02262A
:0738B2000F02261402261983
:10261F009006C2E0FE9006C3E0D39E405F9006C1D5
:10262F00E0B404189006C3E0C395735002D22B9008
:10263F0006C2E0D395734002C22B803E9006C2E0E3
:10264F00C3957350099006C3E0D39573500280026F
:10265F00D22B9006C2E0D3957350099006C3E0C306
:10266F0095735002C22B9006C1E0B401099000D5BA
:10267F00E0D3956150028002C22B802A9006C2E0FF
:10268F00D3957340099006C3E0C39573400280024F
:10269F00C22B9006C2E0C3957340099006C3E0D3E6
:1026AF0095734002D22B229006C5E09038B9F828D6
:1026BF002873804C85537380479000C9E0855FF085
:1026CF00A4FFAEF074081200398F738033856173E5
:1026DF00802E856773802985687380248569738050
:1026EF001F856A73801A856B7380158566738010DA
:1026FF00856573800B856C738006900016E0F5730B
:1038B9000226C10226C30226C80226DC0226E1022C
:1038C90026E60226EB0226F00226F50226FA022651
:0738D900FF0227040227098A
:10270F009006C6E0FE9006C7E0D39E404B9006C5EC
:10271F00E0B404189006C7E0C395735002D22C9012
:10272F0006C6E0D395734002C22C802A9006C6E0FD
:10273F00C3957350099006C7E0D39573500280027A
:10274F00D22C9006C6E0D3957350099006C7E0C30C
:10275F0095735002C22C802A9006C6E0D395734021
:10276F00099006C7E0C3957340028002C22C900601
:10277F00C6E0C3957340099006C7E0D39573400236
:10278F00D22C229006C9E09038E0F8282873804CAC
:10279F0085537380479000C9E0855FF0A4FFAEF0CA
:1027AF0074081200398F738033856173802E8567AB
:1027BF007380298568738024856973801F856A7388
:1027CF00801A856B7380158566738010856573809D
:0C27DF000B856C738006900016E0F5730B
:1038E00002279D02279F0227A40227B80227BD02B4
:1038F00027C20227C70227CC0227D10227D60227D8
:07390000DB0227E00227E5CE
:1027EB009006CAE0FE9006CBE0D39E404B9006C904
:1027FB00E0B404189006CBE0C395735002D22D9031
:10280B0006CAE0D395734002C22D802A9006CAE017
:10281B00C3957350099006CBE0D395735002800299
:10282B00D22D9006CAE0D3957350099006CBE0C326
:10283B0095735002C22D802A9006CAE0D39573403F
:10284B00099006CBE0C3957340028002C22D90061F
:10285B00CAE0C3957340099006CBE0D39573400251
:10286B00D22D229006CDE0903907F8282873804CA2
:10287B0085537380479000C9E0855FF0A4FFAEF0ED
:10288B0074081200398F738033856173802E8567CE
:10289B007380298568738024856973801F856A73AB
:1028AB00801A856B738015856673801085657380C0
:0C28BB000B856C738006900016E0F5732E
:1039070002287902287B022880022894022899023B
:10391700289E0228A30228A80228AD0228B202285E
:07392700B70228BC0228C111
:1028C7009006CEE0FE9006CFE0D39E404B9006CD1B
:1028D700E0B404189006CFE0C395735002D22E904F
:1028E70006CEE0D395734002C22E802A9006CEE032
:1028F700C3957350099006CFE0D3957350028002B9
:10290700D22E9006CEE0D3957350099006CFE0C340
:1029170095735002C22E802A9006CEE0D39573405D
:10292700099006CFE0C3957340028002C22E90063D
:10293700CEE0C3957340099006CFE0D3957340026C
:10294700D22E229006D1E090392EF8282873804C99
:1029570085537380479000C9E0855FF0A4FFAEF010
:1029670074081200398F738033856173802E8567F1
:102977007380298568738024856973801F856A73CE
:10298700801A856B738015856673801085657380E3
:0C2997000B856C738006900016E0F57351
:10392E0002295502295702295C02297002297502C3
:10393E00297A02297F02298402298902298E0229E5
:07394E009302299802299D54
:1029A3009006D2E0FE9006D3E0D39E404B9006D132
:1029B300E0B404189006D3E0C395735002D22F906D
:1029C30006D2E0D395734002C22F802A9006D2E04C
:1029D300C3957350099006D3E0D3957350028002D8
:1029E300D22F9006D2E0D3957350099006D3E0C35B
:1029F30095735002C22F802A9006D2E0D39573407C
:102A0300099006D3E0C3957340028002C22F90065B
:102A1300D2E0C3957340099006D3E0D39573400287
:102A2300D22F229006D5E0903955F8282873804C90
:102A330085537380479000C9E0855FF0A4FFAEF033
:102A430074081200398F738033856173802E856714
:102A53007380298568738024856973801F856A73F1
:102A6300801A856B73801585667380108565738006
:0C2A73000B856C738006900016E0F57374
:10395500022A31022A33022A38022A4C022A51024B
:103965002A56022A5B022A60022A65022A6A022A6C
:073975006F022A74022A7997
:102A7F009006D6E0FE9006D7E0D39E404B9006D549
:102A8F00E0B404189006D7E0C395735002D230908B
:102A9F0006D6E0D395734002C230802A9006D6E066
:102AAF00C3957350099006D7E0D3957350028002F7
:102ABF00D2309006D6E0D3957350099006D7E0C375
:102ACF0095735002C230802A9006D6E0D39573409A
:102ADF00099006D7E0C3957340028002C23090067A
:102AEF00D6E0C3957340099006D7E0D395734002A3
:102AFF00D230229006D9E090397CF8282873804C88
:102B0F0085537380479000C9E0855FF0A4FFAEF056
:102B1F0074081200398F738033856173802E856737
:102B2F007380298568738024856973801F856A7314
:102B3F00801A856B73801585667380108565738029
:0C2B4F000B856C738006900016E0F57397
:10397C00022B0D022B0F022B14022B28022B2D02D3
:10398C002B32022B37022B3C022B41022B46022BF3
:07399C004B022B50022B55DA
:102B5B009006DAE0FE9006DBE0D39E404B9006D960
:102B6B00E0B404189006DBE0C395735002D23190A9
:102B7B0006DAE0D395734002C231802A9006DAE080
:102B8B00C3957350099006DBE0D395735002800216
:102B9B00D2319006DAE0D3957350099006DBE0C38F
:102BAB0095735002C231802A9006DAE0D3957340B8
:102BBB00099006DBE0C3957340028002C231900698
:102BCB00DAE0C3957340099006DBE0D395734002BE
:102BDB00D231229006DDE09039A3F8282873804C7F
:102BEB0085537380479000C9E0855FF0A4FFAEF07A
:102BFB0074081200398F738033856173802E85675B
:102C0B007380298568738024856973801F856A7337
:102C1B00801A856B7380158566738010856573804C
:0C2C2B000B856C738006900016E0F573BA
:1039A300022BE9022BEB022BF0022C04022C09025E
:1039B3002C0E022C13022C18022C1D022C22022C7A
:0739C30027022C2C022C311D
:102C37009006DEE0FE9006DFE0D39E404B9006DD77
:102C4700E0B404189006DFE0C395735002D23290C7
:102C570006DEE0D395734002C232802A9006DEE09A
:102C6700C3957350099006DFE0D395735002800235
:102C7700D2329006DEE0D3957350099006DFE0C3A9
:102C870095735002C232802A9006DEE0D3957340D6
:102C9700099006DFE0C3957340028002C2329006B6
:102CA700DEE0C3957340099006DFE0D395734002D9
:102CB700D232229006E1E09039CAF8282873804C76
:102CC70085537380479000C9E0855FF0A4FFAEF09D
:102CD70074081200398F738033856173802E85677E
:102CE7007380298568738024856973801F856A735B
:102CF700801A856B73801585667380108565738070
:0C2D07000B856C738006900016E0F573DD
:1039CA00022CC5022CC7022CCC022CE0022CE502E8
:1039DA002CEA022CEF022CF4022CF9022CFE022D06
:0739EA0003022D08022D0D60
:102D13009006E2E0FE9006E3E0D39E404B9006E18E
:102D2300E0B404189006E3E0C395735002D23390E5
:102D330006E2E0D395734002C233802A9006E2E0B4
:102D4300C3957350099006E3E0D395735002800254
:102D5300D2339006E2E0D3957350099006E3E0C3C3
:102D630095735002C233802A9006E2E0D3957340F4
:102D7300099006E3E0C3957340028002C2339006D4
:102D8300E2E0C3957340099006E3E0D395734002F4
:102D9300D23322AE2EAF2F74F5D39F74019E400819
:102DA300782E1265E9022EB0752F01752E00AE52F2
:102DB300AF53E546BE000DD39F40099000ABE0D36F
:102DC300954740028023754700E546C39553F57345
:102DD3009000AEE0D395454008E5452573F5458061
:102DE300069000AEE0F54580020547900087E0D3EA
:102DF3009561401CE55FC395604015AE52AF53E546
:102E030046BE00039F50099000ACE0D395484002B2
:102E1300806E9007C7E0A852B8000495535003751D
:102E23004A009007C7E0A852B8000BD39553400659
:102E3300E5539007C7F0E54A7041E553C39546F55E
:102E430073E573D3940540037573059000ADE0C338
:102E530095455007E573C3954540028009E545C391
:102E63009573F54580069000ADE0F5459000ADE023
:102E7300D3954540069000ADE0F5457548008002C6
:102E83000548E54A7016900087E0C39561500DE54B
:102E9300462405A852B8000695534002800F9000BF
:102EA3009AE0F545754A0174789007C7F022AE2E73
:102EB300AF2F74E9D39F74039E4008782E1265E9FF
:102EC30002304F752F01752E00754532A234402A0A
:102ED30075451990009AE075F002A4FFAEF0E5473E
:102EE300BE0006D39F4002D2340547754A03747867
:102EF3009007C7F075490002303EAE52AF53E54626
:102F03006F4E700302303EE546BE000DD39F40096D
:102F13009000ABE0D395474002800F754700E54A28
:102F2300C394035003754519800DE546C39553F5C6
:102F330073E5472573F547900087E0D39561400E0D
:102F43009007C7E0A852B80007D395534002800CFE
:102F5300054990009AE0B54903754A00E54AB40370
:102F630006A20DB3B34002800A0549E549B43C0308
:102F7300754A02E54AB402299007C7E0A852B8008F
:102F83000ED395534009E5539007C7F07549009058
:102F93000087E0C39561500975490074789007C7AD
:102FA300F0E54A705A900087E0D39561401CE55FD5
:102FB300C395604015AE52AF53E546BE00039F5024
:102FC300099000ACE0D3954840028008754800752D
:102FD300454B8028E553C39546F573E573D39405B4
:102FE3004003757305900087E0D395614008E54879
:102FF3002573F5488006E5482406F548754900E53C
:103003004A7016900087E0C39561500DE54624058C
:10301300A852B80006955340028003754A01E54A59
:10302300B40118754519054990009AE0B54906752C
:103033004A0275490074789007C7F0E54575F00AB0
:10304300A4FFAEF09007B8EEF0A3EFF022E56F9087
:1030530039F1F828287390007FE0700302327790EB
:1030630000B5E0B401028003023192900042E0B562
:103073005E02800302318F7E017F00E5BE126595FB
:10308300E5BD2FFF50010E8E5A8F5B7410126595AC
:1030930090006DE08E048F05FF1265859007BCECF0
:1030A300F0A3EDF074FFBC00039D500B74FF900779
:1030B300BCF8E4F0E8A3F0E56B600FE56BC394FEA6
:1030C30050089000DBE06402600280649000C9E075
:1030D300B40B1F9007BCE0FEA3E0FF74E7126595F5
:1030E300E56B8E048F05FF1265859007BCECF0A39A
:1030F300EDF09000C9E0D3940B40089000B1E06478
:10310300046002802B9007BCE0FEA3E0FF9007BEA3
:10311300E0FCA3E0FDEFD39DEE9C400D1265E19032
:1031230007BCEEF0A3EFF080079007BCE4F0A3F038
:1031330090007FE0B4021E9007BCE0FEA3E0FF9086
:1031430007C8E02FFF50010E74011200399007BC2D
:10315300EEF0A3EFF09007BCE0FEA3E0FF9007C8FA
:10316300E0BE0008D39F4004D2378002B2379007F5
:10317300BDE09007C8F09000B1E064016006A2379B
:10318300B3B3400280069007BDE0F55F023275D20B
:10319300377E017F00E5BE126595E5BD2FFF500127
:1031A3000E8E5A8F5B741012659590006DE08E043D
:1031B3008F05FF1265859007BCECF0A3EDF0E56B7E
:1031C300600FE56BC394FE50089000DBE06402607F
:1031D3000280649000C9E0B40B1F9007BCE0FEA31B
:1031E300E0FF74E7126595E56B8E048F05FF1265AA
:1031F300859007BCECF0A3EDF09000C9E0D3940BED
:1032030040089000B1E064046002802B9007BCE0AA
:10321300FEA3E0FF9007BEE0FCA3E0FDEFD39DEE2D
:103223009C400D1265E19007BCEEF0A3EFF0800720
:103233009007BCE4F0A3F090007FE0B4021E900777
:10324300BCE0FEA3E0FF9007C8E02FFF50010E741F
:10325300011200399007BCEEF0A3EFF09007BDE038
:103263009007C8F09000B1E0640160069007BDE0EC
:10327300F55F8003755F0090007BE07006756F015A
:1032830002305075BB1802384590007BE070030292
:1032930033FD7E017F00E5BE126595E5BD2FFF502E
:1032A300010E8E5A8F5B9000C1E0B4010F7E0F7F39
:1032B300FFAC5AAD5B1265E18E5A8F5B9000E6E07E
:1032C300B40245AE5AAF5B90001FE0FCA3E0FDEDF6
:1032D300D39FEC9E400A90001FE55AF0A3E55BF0F4
:1032E300AE5AAF5B900021E0FCA3E0FDEFD39DEE6F
:1032F3009C400A900021E55AF0A3E55BF0AE5AAF7B
:103303005B74041200398F619000E6E0704CAE5A92
:10331300AF5B90001FE0FCA3E0FDEFD39DEE9C406C
:10332300091265E18E5A8F5B8006755B00755A0042
:10333300AE5AAF5B741012659590006AE08E048FED
:1033430005FF1265858C5A8D5B74FFBC0009D39D04
:103353004005855B6180037561FE9000B1E0B401B7
:103363000280030233FBA20DB3B3500E900085E03D
:10337300A852B80005D39553500280719000C2E063
:103383008561F0A4FFAEF074648E048F05FF1265AF
:10339300858C5A8D5BE56B6016E56BC394FE500F0D
:1033A3009000DBE0B402089000C9E0640B60028087
:1033B30017AE5AAF5B74E7126595E56B8E048F0504
:1033C300FF1265858C5A8D5BAE5AAF5B9007BCE0EC
:1033D300FCA3E0FDEDD39FEC9E4005855B5F800B76
:1033E300A237B340069007BDE0F55F800BA237B369
:1033F30040069007BDE0F55F800375610090007E95
:10340300E07006756F0202305075BB1902384590A3
:10341300007EE070030234B2E55ED39551400302AF
:1034230034B090001DE0FEA3E0FFE5651265D9907E
:10343300001DEEF0A3EFF07E017F00E5BE1265955F
:10344300E5BD2FFF50010E8E5A8F5B9000EBE070AD
:1034530013740A12659574518E048F05FF126585E6
:103463008D658019AE5AAF5B740A1265958F048E11
:10347300057E017F95CDCCCD1264838F65E565D341
:103483009464400375656490001DE0FEA3E0FFE5CE
:10349300652FFF50010E90001DEEF0A3EFF090009A
:1034A30082E0048E048F05FF1265858D65800375A8
:1034B30065329000CEE07006756F0302305075BB25
:1034C300130238459000CEE0604A7E017F00E5BEDE
:1034D300126595E5BD2FFF50010E8E5A8F5B740464
:1034E3001200398F669000D0E08566F0A4FDACF041
:1034F3007464FF1265858D669000CFE08566F0A445
:10350300FFAEF074FF8E048F05FF126585ED90000A
:1035130069F0800375660090007CE07006756F04A7
:1035230002305075BB1702384590007CE0B40102AD
:1035330080030235C07E017F00E5BE126595E5BDBF
:103543002FFF50010E8E5A8F5B9007C9E0601990D0
:1035530007C9E014905EF512008CE493FC740193A8
:10356300FDEDC39FEC9E400280069007C9E014F076
:103573009007C9E0C394B3501DAE5AAF5B9007C91F
:10358300E004905EF512008CE493FC740193FDEF6C
:10359300C39DEE9C400280069007C9E004F09007AB
:1035A300C9E0FE9000A2E08E0088F0A4FFAEF074A4
:1035B300648E048F05FF1265858D67800375670030
:1035C30090007DE07006756F0502305075BB1602E2
:1035D300384590007DE0B4010280030236697E0124
:1035E3007F00E5BE126595E5BD2FFF50010E8E5A93
:1035F3008F5B9007CAE060199007CAE01490605F80
:1036030012008CE493FC740193FDEDC39FEC9E4088
:103613000280069007CAE014F09007CAE0C394B38F
:10362300501DAE5AAF5B9007CAE00490605F120072
:103633008CE493FC740193FDEFC39DEE9C400280E8
:10364300069007CAE004F09007CAE0FE9000A8E0E5
:103653008E0088F0A4FFAEF074648E048F05FF1211
:1036630065858D68800375680075BB1F0238457ECC
:10367300017F00E5BE126595E5BD2FFF50010E8E5B
:103683005A8F5B740912659574E68E048F05FF12D9
:1036930065858D6A900084E07006756F070230506F
:1036A30075BB15023845900084E070030237C47E71
:1036B300017F00E5BE126595E5BD2FFF50010E8E1B
:1036C3005A8F5B74041200398F69900084E0B4014F
:1036D300159000D8E08569F0A4FFAEF074071200DE
:1036E30039EF9007C1F0900084E0B402159000D840
:1036F300E08569F0A4FFAEF07407120039EF90077C
:10370300C0F0900084E0B4030280030237A7900066
:10371300C5E0701CE569C394195002D229E569D349
:1037230094644002C2299000A4E09007C4F080632F
:103733009000A4E070349000D8E08569F0A4FFAE57
:10374300F074FF8E048F05FF126585ED9007C4F0BA
:10375300AE52AF53741EBE0006D39F4002D229E57A
:1037630061D394E54002C2298029E569C3940A50D4
:103773000DAE52AF53741EBE0004D39F500280029D
:10378300D229E561D394E54002C2299000A4E090D8
:1037930007C4F09007C4E0C394055006740590076E
:1037A300C4F0C238900084E0B40414E569C39419EA
:1037B3005002D238E569D394324002C238C229801C
:1037C300037569009000DBE07006756F08023050E6
:1037D30075BB14806D9000DBE060567E017F00E5D1
:1037E300BE126595E5BD2FFF50010E8E5A8F5BEF1C
:1037F300D39421EE940E4005756BFF8015AE5AAF3E
:103803005B741012659574E38E048F05FF12658552
:103813008D6BE56B75F00BA4FFAEF09000C9E08EE5
:10382300048F05FF1265859007BEECF0A3EDF080D1
:1038330003756B0090007FE0600575BB1A8003750C
:02384300BB18B0
:1039F10002305902328C0234120234C702352C02D1
:0B3A010035D50236720236A90237D814
:05384500056FD2EC222A
:0965C7002582F5825002058322B1
:0F008C0025E050020583258250020583F582226C
:10656400EF2F500205832582F582E5833E2EF583C5
:016574002204
:1065D900CFC39FFF50011E22C3EF9DFFEE9CFE22F9
:0865E9000806B60002180622A4
:0D65A300A3E004F07006120049E004F022AD
:0E003900048007C3CE13CECF13CFD5E0F6223E
:10648300BC000FBE0008ED8FF084FFADF022E4FEE8
:10649300FF22BE000DEF60FE54F0606F20E70302A1
:1064A3006539EAC0E0EBC0E078017A0075F001EEEF
:1064B30020E710EF25E0FFEE33FE0AC5F023C5F019
:1064C30030E7F0EA5407F9096A7A007B00600108B3
:1064D300C3EC9E40167004ED9F4010ED9FFDEC9EB3
:1064E300FCE5F0CA4ACA03F5F08005E5F003F5F0D0
:1064F300C3EE13FEEF13FFD9D77908CACBCAD8D09E
:10650300EAFEEBFFD0E0FBD0E0FA22EC8FF084FC54
:10651300ED54F045F0C48FF084FEEDC454F045F023
:10652300C48FF084FDEEC4FE54F02DFFEE540F3CF7
:10653300FEADF07C0022790078008FF0EC7E08201D
:10654300E70DC3CD33CD33C933C9C833C8DEF084B7
:1065530049F9E5F08FF0BE00E6FD7C00E9FFE8FEB7
:016563002215
:0E659500F88FF0A4FFE5F0CE88F0A42EFE22D1
:10000300EF8DF0A4F9A8F0EF8CF0A428F8EE8DF0B2
:06001300A428FEE9FF2213
:10657500600D782B02657F007830D8FED5E0F822D3
:10658500EEC0E07E00126483EFFDEEFCD0E0FE225B
:0C65B000EEC0E07E00126483D0E0FE220A
:03001B0002001EC2
:0300530002005652
:03009B00020071EF
:030000000265D0C6
:0965D00075817575D0000242B11D
:0B65BC00E5822FF582E5833EF5832287
:0A0049000582D5820215831582227C
:10001E00C0E0C0F0C083C082C0D075D0001241EBEA
:0B002E00D0D0D082D083D0F0D0E032E0
:10005600C0E0C0F0C083C082C0D075D0001241EEAF
:10006600D0D0D082D083D0F0D0E032C0E0C0F0C093
:1000760083C082C0D075D000124273D0D0D082D057
:0600860083D0F0D0E0324F
:00000001FF
